:020000020000FC
:100000000C94694318951895189518951895189596
:100010001895189518951895189518951895189578
:100020001895189518951895189518951895189568
:100030001895189518951895189518950C94CB3215
:1000400018951895189518950C94E64018951895DC
:100050001895189518951895189518951895189538
:100060001895189518951895189518951895189528
:1000700018951895189518950C94C14018951895D1
:100080001895189518951895189518950D0A20002B
:100090000D0A0A205B434D322056657273696F6EFC
:1000A00020312E315D000D0A20546F7373204D6F87
:1000B00064650D0A000D0A202D3E5B44796E616D6A
:1000C0006978656C5D3A000D0A203C2D5B44796EC1
:1000D000616D6978656C5D3A000D0A2052533233C8
:1000E000323A00202052533438353A000D0A20416C
:1000F000726520796F752073757265203F28792F9E
:100100004E29000D0A205573616765203A20476F1C
:10011000205B506F736974696F6E20416E676C6508
:1001200028307830307E3078336666295D000D0ADD
:1001300020416C6C2044796E616D6978656C277321
:100140002049442077696C6C2062652073657420B7
:10015000746F203078002E2041726520796F7520F1
:10016000737572653F28592F4E29000D0A2045727C
:10017000726F72315B436865636B2044796E616DA9
:100180006978656C2056657273696F6E206973209B
:100190006D6F7265207468616E20335D000D0A20FA
:1001A00042286265666F7265292C4E286E657874E8
:1001B000292C51285175697429000D0A20343835CD
:1001C0004D6F6E69746F72205B4C462C43522061F8
:1001D0007265206164646564206174207061757368
:1001E000652074696D655D0D0A000D0A204E6F2053
:1001F000446174615B61742042726F616463617316
:100200007420494420307846455D000D0A204E6F29
:10021000204461746128436865636B2049442C2045
:100220004F7065726174696E67204D6F64652C2034
:100230004261756420726174652900284C454E3A0C
:10024000000D0A204C454420426C696E6B204944E5
:100250003A3058002044796E616D6978656C73207E
:10026000466F756E642E000D0A204C454420426C8A
:10027000696E6B2049443A3058000D20466F756E08
:100280006421202D2D20424155445F5245473A308C
:1002900078002C2049443A3078000D0A20426175DC
:1002A000642052617465206973206368616E6765BC
:1002B0006420746F2000425053000D0A2049443AD4
:1002C00030783030202D20000D0A2044656C617993
:1002D0003A000D0A20546F7271756520456E616297
:1002E0006C65000D0A204D6F766520307830303017
:1002F00030203C2D3E20307830336666000D0A20D9
:10030000416E79204B657920746F20436F6E74695C
:100310006E75652E2E2E000D0A205B454550524FFE
:100320004D20415245415D0D0A204D4F44454C5FE3
:100330004E554D4245525F4C202020202020202049
:10034000285229205B000D0A204D4F44454C5F4E3A
:10035000554D4245525F4820202020202020202853
:100360005229205B000D0A2056455253494F4E201A
:100370002020202020202020202020202020285243
:1003800029205B000D0A2049442020202020202025
:1003900020202020202020202020202028522F57DD
:1003A000295B000D0A20424155445F5241544520CB
:1003B000202020202020202020202028522F5729B4
:1003C0005B000D0A2052455455524E5F44454C4146
:1003D000595F54494D452020202028522F57295B32
:1003E000000D0A2043575F414E474C455F4C494D35
:1003F00049545F4C202020202028522F57295B0091
:100400000D0A2043575F414E474C455F4C494D49CB
:10041000545F48202020202028522F57295B000DB0
:100420000A204343575F414E474C455F4C494D4975
:10043000545F4C2020202028522F57295B000D0AA2
:10044000204343575F414E474C455F4C494D49540B
:100450005F482020202028522F57295B000D0A20BA
:10046000285245534552564544292020202020201B
:10047000202020202028522F57295B000D0A204CD5
:10048000494D49545F54454D50455241545552458C
:100490002020202028522F57295B000D0A20444F8E
:1004A000574E5F4C494D49545F564F4C5441474558
:1004B00020202028522F57295B000D0A2055505F1D
:1004C0004C494D49545F564F4C54414745202020DC
:1004D000202028522F57295B000D0A204D41585FDC
:1004E000544F525155455F4C202020202020202081
:1004F0002028522F57295B000D0A204D41585F5488
:100500004F525155455F4820202020202020202098
:1005100028522F57295B000D0A2052455455524E40
:100520005F4C4556454C20202020202020202028AC
:10053000522F57295B000D0A20414C41524D5F4C10
:100540004544202020202020202020202020285228
:100550002F57295B000D0A20414C41524D5F5348F3
:100560005554444F574E2020202020202028522F21
:1005700057295B000D0A20285245534552564544E1
:1005800029202020202020202020202028522F57E2
:10059000295B000D0A20444F574E5F43414C4942AE
:1005A000524154494F4E5F4C20202028522F57294A
:1005B0005B000D0A20444F574E5F43414C49425265
:1005C0004154494F4E5F4820202028522F57295B25
:1005D000000D0A2055505F43414C49425241544955
:1005E0004F4E5F4C202020202028522F57295B009F
:1005F0000D0A2055505F43414C4942524154494FE6
:100600004E5F48202020202028522F57295B000DC4
:100610000A205B52414D20415245415D0D0A205454
:100620004F525155455F454E41424C4520202020B8
:100630002020202028522F57295B000D0A204C45EE
:100640004420202020202020202020202020202086
:1006500020202028522F57295B000D0A2043575F86
:10066000434F4D504C49414E43455F4D41524749E0
:100670004E2028522F57295B000D0A204343575F15
:10068000434F4D504C49414E43455F4D41524749C0
:100690004E28522F57295B000D0A2043575F434FC6
:1006A0004D504C49414E43455F534C4F50452020DF
:1006B00028522F57295B000D0A204343575F434FB1
:1006C0004D504C49414E43455F534C4F50452028B7
:1006D000522F57295B000D0A20474F414C5F504F66
:1006E000534954494F4E5F4C20202020202028524F
:1006F0002F57295B000D0A20474F414C5F504F5345
:100700004954494F4E5F4820202020202028522F56
:1007100057295B000D0A204D4F56494E475F5350F5
:100720004545445F4C2020202020202028522F5770
:10073000295B000D0A204D4F56494E475F535045E7
:1007400045445F482020202020202028522F572970
:100750005B000D0A20544F525155455F4C494D499D
:10076000545F4C2020202020202028522F57295B26
:10077000000D0A20544F525155455F4C494D495484
:100780005F482020202020202028522F57295B005E
:100790000D0A2050524553454E545F504F53495413
:1007A000494F4E5F4C20202020285229205B000D0D
:1007B0000A2050524553454E545F504F53495449B7
:1007C0004F4E5F4820202020285229205B000D0A30
:1007D0002050524553454E545F53504545445F4C5D
:1007E00020202020202020285229205B000D0A20D4
:1007F00050524553454E545F53504545445F482041
:10080000202020202020285229205B000D0A205083
:10081000524553454E545F4C4F41445F4C2020207D
:100820002020202020285229205B000D0A20505231
:100830004553454E545F4C4F41445F482020202093
:1008400020202020285229205B000D0A20505245EC
:1008500053454E545F564F4C54414745202020206D
:10086000202020285229205B000D0A205052455399
:10087000454E545F54454D504552415455524520C4
:100880002020285229205B000D0A20524547495359
:1008900054455245445F494E5354525543202020FD
:1008A00028522F57295B000D0A20524553455256B6
:1008B00045442850415553455F54494D452920280A
:1008C000522F57295B000D0A204D4F56494E4720A5
:1008D0002020202020202020202020202020202810
:1008E0005229205B000D0A204C4F434B2020202032
:1008F0002020202020202020202020202028522FAF
:1009000057295B000D0A2050554E43485F4C20206C
:1009100020202020202020202020202028522F5757
:10092000295B000D0A2050554E43485F4820202087
:10093000202020202020202020202028522F57292E
:100940005B000D0A0A202044554D50284429203AC6
:100950002044756D7020636F6E74726F6C207461CB
:10096000626C652E000D0A20204944205B49445FDB
:100970004E554D5D203A20536574204944206F66E2
:100980002064796E616D6978656C2E000D0A2020F7
:10099000434944205B49445F4E554D5D203A204316
:1009A00068616E676520436F6E74726F6C20494496
:1009B0002E000D0A202052454144205B4144445200
:1009C0005D5B4C454E5D203A205265616420646158
:1009D00074612E206578295265616420313020329F
:1009E0002028526561642066726F6D203078313046
:1009F0002C206C656E677468203229000D0A202057
:100A00005752495445205B414444525D5B44415434
:100A100041315D2E2E203A20577269746520646141
:100A200074612E2065782957726974652031342CE1
:100A30003120285772697465203120617420307824
:100A4000313429000D0A20205245475F5752205B60
:100A5000414444525D5B44415441315D2E2E203A65
:100A600020526567697374657220777269746520B6
:100A7000696E737475726374696F6E000D0A20205D
:100A8000414354494F4E203A20416374696F6E20B0
:100A90005245475F575220696E737472756374696B
:100AA0006F6E000D0A2020476F205B504F53495452
:100AB000494F4E5D5B53504545445D3A20476F7446
:100AC0006F2074686520706F736974696F6E20772A
:100AD000697468207468652073706565642E000D04
:100AE0000A2020484558205B4E554D5D5B4E554DC4
:100AF0005D2E2E2E203A205472616E736D697465DE
:100B00002072617720646174612E206578294865C0
:100B100078204646204646203031203033000D0AEA
:100B200020205245534554203A2044796E616D6926
:100B300078656C2052657365742E000D0A20205074
:100B4000494E47205B4E554D5D3A2065782920502F
:100B5000696E67204E554D2049442064796E616D61
:100B60006978656C2E000D0A2020535752205B4196
:100B70004444525D5B4C454E5D5B49445D5B444182
:100B800054415D2E2E2E5B49445D5B444154415DD2
:100B90002E2E2E203A2053796E6320577269746589
:100BA0002E000D0A20205343414E205B4E554D5DD3
:100BB000203A205343414E206C696E6B656420647B
:100BC000796E616D6978656C20696E20307E4E5556
:100BD0004D20696E2063757272656E742062617556
:100BE0006420726174652E000D0A20204C4544205B
:100BF0005B4E554D5D203A20426C696E6B204C4532
:100C000044206F66204E554D2049442E2027422710
:100C10002C274E2720666F72204944206368616E3E
:100C200067652E2027512720666F722051756974E1
:100C30002E000D0A202042415544205B4E554D5D4B
:100C4000203A205365742062617564207261746576
:100C500020206578292042415544203232283537FA
:100C6000363030425053292C2042415544203128FF
:100C7000314D42505329000D0A2020534541524323
:100C800048203A2053656172636820494420616EB0
:100C900064206261756472617465206F6620616CA6
:100CA0006C206C696E6B65642064796E616D697827
:100CB000656C732E000D0A202055706461746520E8
:100CC0005B53544152545F49445D205B454E445F41
:100CD00049445D203A2044796E616D6978656C20E5
:100CE0006669726D77617265207570646174652ED6
:100CF0002873797374656D2075736572206F6E6CDF
:100D00007929000D0A0A20202020202020202043BD
:100D10006F7079726967687420524F424F5449531B
:100D200020434F2E2C4C54442E0D0A000D0A205304
:100D30006572766F20436865636B0D0A000D0A20AB
:100D40003078002044584C732061726520666F75BE
:100D50006E642E202D534552564F5F4E554D3A30FE
:100D600078005B496E76616C69642050616765202C
:100D7000526561643A000D0A205B4572726F723AE7
:100D80005278442054696D656F75745D000D0A20BA
:100D90005B4572726F723A57726F6E672048656179
:100DA0006465725D000D0A205B4572726F723A5481
:100DB00078494420213D20527849445D000D0A20A5
:100DC0005B4572726F723A57726F6E67204C656E38
:100DD0006774685D000D0A205B4572726F723A5746
:100DE000726F6E6720436865636B53756D5D000DB0
:100DF0000A20555044415445205B535441525420DD
:100E000049445D205B454E442049445D00295D3ADC
:100E100000283078000D0A2049443A0020537461BC
:100E20006E6462792E002057726974696E672E2E87
:100E30000020537563636573732E00204572726FD3
:100E4000722E000D0A204572722049443A30780013
:100E50002042616420436F6D6D616E640041540DEA
:100E60000A000D0A2053657269616C204361626C4F
:100E70006520506C7567206F75742C20616E64203E
:100E8000507573682074686520627574746F6E00A5
:100E900041542B4254494E464F3F0D0A000D0A2043
:100EA000426C7565546F6F74682041646472657339
:100EB000733A000D0A2053572050757368656428F3
:100EC000546F72717565204F464629000D0A2049FE
:100ED0006E697469616C20506F736974696F6E20FC
:100EE000776173206E6F7420496E697469616C69F3
:100EF0007A65642E28546F72717565204F464629B5
:100F00000041542B55415254434F4E4649472C35CE
:100F1000373630302C4E2C310D0A000D0A2050751A
:100F2000736820627574746F6E207768656E2072C6
:100F3000656164792E2E2E000D0A205550205B53DA
:100F4000544152545D205B4C454E4754485D005B14
:100F5000457869745D000D44796E616D6978656CE2
:100F60002049442030783030205B202020205D2034
:100F70002020202020202020202020202020202071
:100F80002020202020202020202020202020202061
:100F90002020202020000D0A44796E616D6978655B
:100FA0006C2049442030783031205B202020205DA7
:100FB0002020202020202020202020202020202031
:100FC0002020202020202020202020202020202021
:100FD00020202020202020506167654E756D6265BD
:100FE000723A000D0A44796E616D6978656C20492A
:100FF000442030783032205B202020205D202020CB
:1010000020202020202020202020202020202020E0
:1010100020202020202020202020202020202020D0
:1010200020202020416464723A000D0A44796E61E8
:101030006D6978656C2049442030783033205B201E
:101040002020205D20202020202020202020202063
:101050002020202020202020202020202020202090
:101060002020202020202020202020285265736569
:10107000727665642920203A000D0A44796E616D0C
:101080006978656C2049442030783034205B20201A
:1010900020205D2020202020202020202020202013
:1010A0002020202020202020202020202020202040
:1010B00020202020202020202020285265736572C7
:1010C0007665642920203A000D0A44796E616D69C5
:1010D00078656C2049442030783035205B20202012
:1010E000205D2020202020202020202020202020C3
:1010F00020202020202020202020202020202020F0
:101100002020202020202020202852657365727620
:1011100065642920203A000D0A44796E616D697872
:10112000656C2049442030783036205B2020202018
:101130005D20202020202020202020202020202072
:10114000202020202020202020202020202020209F
:10115000202020202020202028526573657276658B
:10116000642920203A000D0A44796E616D69786522
:101170006C2049442030783037205B202020205DCF
:10118000202020202020202020202020202020205F
:10119000202020202020202020202020202020204F
:1011A00020202020202020285265736572766564F7
:1011B0002920203A000D0A44796E616D6978656CCA
:1011C0002049442030783038205B202020205D20CA
:1011D000202020202020202020202020202020200F
:1011E00020202020202020202020202020202020FF
:1011F000202020202020285265736572766564299E
:1012000020203A000D0A44796E616D6978656C2082
:1012100049442030783039205B202020205D202078
:1012200020202020202020202020202020202020BE
:1012300020202020202020202020202020202020AE
:1012400020202020202020205061676520537465D5
:10125000703A000D0A44796E616D6978656C2049B9
:10126000442030783041205B202020205D20202049
:10127000202020202020202020202020202020206E
:10128000202020202020202020202020202020205E
:1012900020202020436F6E74726F6C20436F646552
:1012A0003A000D0A44796E616D6978656C20494495
:1012B0002030783042205B202020205D202020201C
:1012C000202020202020202020202020202020201E
:1012D000202020202020202020202020202020200E
:1012E0002020202020506167652053706565643A96
:1012F000000D0A44796E616D6978656C204944205F
:1013000030783043205B202020205D2020202020CA
:1013100020202020202020202020202020202020CD
:1013200020202020202020202020202020202020BD
:10133000202020202044584C2053657475703A00BA
:101340000D0A44796E616D6978656C2049442030DE
:10135000783044205B202020205D20202020202089
:10136000202020202020202020202020202020207D
:10137000202020202020202020202020202020206D
:10138000202020416363656C2054696D653A000D2F
:101390000A44796E616D6978656C20494420307823
:1013A0003045205B202020205D2020202020202090
:1013B000202020202020202020202020202020202D
:1013C000202020202020202020202020202020201D
:1013D0004C696E6B20746F204E6578743A000D0A6C
:1013E00044796E616D6978656C20494420307830AD
:1013F00046205B202020205D20202020202020204F
:1014000020202020202020202020202020202020DC
:101410002020202020202020202020202020204CA0
:10142000696E6B20746F20457869743A000D0A4428
:10143000796E616D6978656C20494420307831306F
:10144000205B202020205D20202020202020202024
:10145000202020202020202020202020202020208C
:101460002020202020202020202020202020285242
:10147000657365727665642920203A000D0A447907
:101480006E616D6978656C20494420307831312077
:101490005B202020205D20202020202020202020D4
:1014A000202020202020202020202020202020203C
:1014B00020202020202020202020202020285265AD
:1014C0007365727665642920203A000D0A44796EAE
:1014D000616D6978656C2049442030783132205B39
:1014E000202020205D2020202020202020202020BF
:1014F00020202020202020202020202020202020EC
:101500002020202020202020202020202852657309
:1015100065727665642920203A000D0A44796E616F
:101520006D6978656C2049442030783133205B2028
:101530002020205D2020202020202020202020206E
:10154000202020202020202020202020202020209B
:101550002020202020202020202020285265736574
:10156000727665642920203A000D0A44796E616D17
:101570006978656C2049442030783134205B202024
:1015800020205D202020202020202020202020201E
:10159000202020202020202020202020202020204B
:1015A00020202020202020202020472C572C492C90
:1015B000442C4D2C536574000D0A44796E616D699D
:1015C00078656C2049442030783135205B2020201C
:1015D000205D2020202020202020202020202020CE
:1015E00020202020202020202020202020202020FB
:1015F000202020202020202020502C4E2C422C4324
:101600006F70792C53617665000D0A44796E616DB7
:101610006978656C2049442030783136205B202081
:1016200020205D202020202020202020202020207D
:1016300020202020202020202020202020202020AA
:10164000202020202020202020204F6E2C4F666656
:101650002C4E65772C5350000D0A202020506175C8
:10166000736554696D65202020202020205B202098
:101670005D2020202020202020202020202020202D
:10168000202020202020202020202020202020205A
:10169000202020202020202020496E632C446563D8
:1016A0003A5D5B2C7D7B000D0A2020205370656520
:1016B0006420202020202020202020205B20205D6E
:1016C000202020202020202020202020202020201A
:1016D000202020202020202020202020202020200A
:1016E00020202020205B583A2D2D2C593A2D2D2CCE
:1016F000413A2D2D2D2D5D000D0A20202020202087
:101700002020202020202020202020202053545042
:1017100037202053545030205354503120535450CC
:1017200032205354503320535450342053545035A6
:10173000205354503620202020476F20537465706A
:101740003A2020202020000D0A20202020202020C8
:101750002020202020202020202020205B20205D11
:101760002020202020202020202020202020202079
:101770002020202020202020202020202020202069
:101780002020202020202020496E632C4465633ACD
:101790005D5B2C7D7B000D0A202020546F727175DB
:1017A00065204C696D6974202020205B20205D201D
:1017B0002020202020202020202020202020202029
:1017C0002020202020202020202020202020202019
:1017D000202020205B583A2D2D2C593A2D2D2C41BC
:1017E0003A2D2D2D2D5D000D0A20202020202020B7
:1017F00020202020202020202020202020202020E9
:1018000020204D53545220534C4156204F465354A0
:1018100020534554302053455431205345543220F1
:101820005345543320202020476F20537465703A6D
:101830002020202020000D0A5D205F202020202075
:101840002020202020202020202020202020202098
:101850002020202020202020202020202020202088
:101860002020202020202020202020202020202078
:101870002020202020202020202020202020202068
:1018800020202020002041726520796F752073751B
:1018900072653F5B792F4E5D0020496E76616C6901
:1018A0006420506167650020496E76616C69642030
:1018B000506172616D6574657200204F6666736574
:1018C00074205570646174656400204F7574206FD6
:1018D000662052616E676500204F4B0003404B4508
:1018E0004D4840454A1B0102030A1A191919010102
:1018F00001010101010101010101010101010101D8
:1019000001010101010000000101010200020001CA
:1019100001010102000101010102000200010101B7
:1019200001010102000200020002000200020001A7
:0D193000010101010102000101020002009D
:10193E00682FA901812F0023B9F40FE003BF00E047
:10194E0002BF09E01DE30E94C14310E0003021E018
:10195E00120710F000E009C001BF082F00FB07B707
:10196E0001F907BF01E001C000E0862F08959A93A8
:10197E008A93902F80E00DC01E981C981B9804E649
:10198E0010E07CD01E9A1C9A1B9A0CE211E076D0C5
:10199E008395891788F300E911E070D089919991A8
:1019AE0008950CC01E981C981B9804E610E066D093
:1019BE001E9A1C9A1B9A04E610E060D00D99F2CF85
:1019CE001E981C981B980D9BFECF1E9A1C9A1B9A54
:1019DE00089500E00093610002B901BB04BB07BB90
:1019EE000ABB00E0009365000093620003B902BBDE
:1019FE0005BB08BB00B50B7F00BD1D9A949ADE9AFD
:101A0E00B89A02B10C6D02B9C09A1F9A1E9A1C9A0E
:101A1E001B9A0895002391F400E00093900019B9E9
:101A2E0002E00BB908E10AB920FB0EF4579A06E062
:101A3E00009395000FEF0CB95E9A08950130E9F40A
:101A4E0000E0009398001093990002E000939B0031
:101A5E0008E100939A0020FB2EF400919A00006892
:101A6E0000939A0006E000939D000FEF00939C00F8
:101A7E0000919B00006400939B000895592F482FFE
:101A8E0080E090E008C02FE93FE021503040E9F7B8
:101A9E0000C00000019680179107A8F3842F952FA0
:101AAE0008955E9A1A9A2CD05E9BFECF1A980895CE
:101ABE008A93802F082F02950F70005D0A3308F06D
:101ACE00095F22D08F70805D082F0A3308F0095FFE
:101ADE001BD000E219D0899108958A93802F082F88
:101AEE0002950F70005D0A3308F0095F0DD08F70FC
:101AFE00805D082F0A3308F0095F06D0899108959A
:101B0E005D9BFECF0CB9089510919B00212F25FFF0
:101B1E00FBCF00939C0008959A938A93802F082FF1
:101B2E0044E60E949743902F092F005DEDDF04E6F7
:101B3E00909F8019082F4AE00E949743902F092FFB
:101B4E00005DE2DF0AE0909F8019805D082FDCDFE8
:101B5E008991999108950E94574448015901DD24B5
:101B6E00BB2052F49094A094B094000B8194900AF0
:101B7E00A00AB00A0DE2C8DF80E09AECAAE9BBE346
:101B8E00CC241AC0DD2019F08201005DBDDF820178
:101B9E009301AC01BD010E94E643801A910AA20A8C
:101BAE00B30A8C019D014AE050E060E070E00E94B3
:101BBE003044C801D901C39409E0C016A8F48401C9
:101BCE009501AC01BD010E943044402E552466247F
:101BDE007724042D052906290729A1F28201005D2B
:101BEE0093DFDD24D394D3CF84019501AC01BD01E5
:101BFE000E943044402E552466247724042D005D27
:101C0E0083DFEEE00C9466449A938A93C8018C01AC
:101C1E00012F10E062DF082F60DF899199910895FE
:101C2E000E946144C801D9018C019D01022F132F1E
:101C3E00330F220B330BE8DF8C01E6DFE4E00C946C
:101C4E007044BA93AA93D80103C00C915DDF11962C
:101C5E000C910023D1F7A991B991089500919B00A1
:101C6E00102F17FFFBCF00919C00089510936F0962
:101C7E0011E01093700922E012E00E9451420023FD
:101C8E0019F00091D80908950FEF089510936F0978
:101C9E0012E01093700922E012E00E9451420023DC
:101CAE0049F03091D90920E00091D80910E0020FD7
:101CBE00131F08950FEF1FEF089510936F092093D0
:101CCE00700922E013E00E945142089510936F09AB
:101CDE002093700922E013E00E94D54108951093DD
:101CEE006F09122F10937009232F30E02093710982
:101CFE0023E013E00E94D54108950E945844EF97C7
:101D0E00E397D2501B98CC2401E00093A90A0093CC
:101D1E00AA0A00E00093660E21C090E0FC01E95C87
:101D2E00F54F0081EDDE5E9A839590E0E82DF0E0B0
:101D3E0031978E179F078CF35E9BFECF1A980FEF8D
:101D4E000E9435410093AB0A07EC10E00E94EF426F
:101D5E002091AB0A03ED19E00E942442CC2011F031
:101D6E000C942B1803EC17E06CDF00919C0AB5DE87
:101D7E000EEC17E066DF20E08E0108571F4F0E9421
:101D8E00252300E00883AE0148575F4F9E01205F78
:101D9E003F4F8E010E94D921802E0091A70A0093F9
:101DAE00A80A8820D9F20FE1801610F00EE1802EDD
:101DBE0025ED37E08E010E94B721002339F421ED85
:101DCE0037E08E010E94B721002359F00FEF2FEF5D
:101DDE003FE0A9010E94934308E001BD04E610E034
:101DEE004DDE27EE36E08E010E94B721002339F436
:101DFE002BEE36E08E010E94B721002361F105EB38
:101E0E0010E00E94EF4280E01CC0FE017096082F89
:101E1E0010E0000F111F000F111FE00FF11F0081C6
:101E2E0011812281338190E0FC01E95CF54F008342
:101E3E0090E0FC01E95CF54F00814FDE00E264DECC
:101E4E00839590E0E82DF0E031978E179F07ECF226
:101E5E001A9A80E06ACF2DEE36E08E010E94B721ED
:101E6E00002371F422EF36E08E010E94B721002389
:101E7E0039F425EF36E08E010E94B721002399F048
:101E8E00088919892A893B8900936F090C891D8954
:101E9E002E893F890093700922E012E000919C0A7E
:101EAE000E9451425BCF27EF36E08E010E94B72190
:101EBE000023A1F014E300919C0AE8DEC801282F4C
:101ECE0014E100919C0A0E946721892F90E0282F2F
:101EDE0015E100919C0A0E94672140CF2CEF36E05D
:101EEE008E010E94B7210023A1F014E300919C0AF9
:101EFE00CDDEC801282F16E100919C0A0E946721B1
:101F0E00892F90E0282F17E100919C0A0E946721EB
:101F1E0025CF21E037E08E010E94B721002339F44E
:101F2E0025E037E08E010E94B7210023F9F080E012
:101F3E0014C0FE017096082F10E0000F111F000F45
:101F4E00111FE00FF11F008111812281338190E07A
:101F5E00FC01E159F64F00838395881550F38A945E
:101F6E00282D13E80EEF0E945142F8CE2DE037E0F7
:101F7E008E010E94B721002371F423E137E08E0118
:101F8E000E94B721002339F42CEF37E08E010E9416
:101F9E00B721002301F180E014C0FE017096082FD6
:101FAE0010E0000F111F000F111FE00FF11F008135
:101FBE0011812281338190E0FC01E159F64F0083BB
:101FCE008395881550F38A94282D13E000919C0A6E
:101FDE000E945142C3CE2EEF37E08E010E94B721F0
:101FEE00002339F425E038E08E010E94B72100234A
:101FFE0001F180E014C0FE017096082F10E0000F72
:10200E00111F000F111FE00FF11F0081118122819E
:10201E00338190E0FC01E159F64F008383958815DA
:10202E0050F38A94282D14E000919C0A0E9451428C
:10203E0095CE29E038E08E010E94B721002339F4B5
:10204E0020E138E08E010E94B7210023F9F080E0F4
:10205E0014C0FE017096082F10E0000F111F000F24
:10206E00111FE00FF11F008111812281338190E059
:10207E00FC01E159F64F00838395881550F38A943D
:10208E00282D15E00EEF0E94514268CE24E138E073
:10209E008E010E94B721002381F00C891D892E89A3
:1020AE003F89202F488959896A897B898A01102F97
:1020BE0000919C0A0E94672151CE2BE138E08E01DF
:1020CE000E94B721002339F10CEE10E00E94EF427E
:1020DE00C5DD093719F0093509F040CE01E080164B
:1020EE0019F400919C0A04C0088919892A893B8930
:1020FE0020E016E00E945142002309F42FCE01E2A7
:10210E0018E09FDD01E000939C0A21E030E0A90178
:10211E000E94934323CE2CE238E08E010E94B72119
:10212E000023A1F001E0801639F420E017E00091C1
:10213E009C0A0E94514212CE20E017E0488959892C
:10214E006A897B89042F0E94514208CE23E338E02E
:10215E008E010E94B721002339F426E338E08E0168
:10216E000E94B7210023D9F102E0801619F003E096
:10217E00801681F50EE100936F09088919892A8965
:10218E003B8900937009088919892A893B89012F97
:10219E0010E00093710903E08016A9F40C891D89E3
:1021AE002E893F89009372090C891D892E893F89DA
:1021BE00012F10E00093730925E013E000919C0AB3
:1021CE000E945142CBCD23E013E000919C0A0E9465
:1021DE005142C4CD03E011E00E94EF42BFCD28E38F
:1021EE0038E08E010E94B721002359F101E08016DC
:1021FE0019F400919C0A04C0088919892A893B891F
:10220E0020E011E00E94D541802F05EB10E00E94E6
:10221E00EF42282F07E31AE00E9424420FEF10E04E
:10222E002DDC0FEF0E9435410093AB0A07EC10E056
:10223E000E94EF422091AB0A03ED19E00E94244266
:10224E008DCD2DE338E08E010E94B721002339F4A5
:10225E0022E438E08E010E94B7210023F1F001E064
:10226E00801611F4A0E805C0088919892A893B89CE
:10227E00A02F80E0833008F071CD0FEF41DC05E533
:10228E003FDC0A2F3DDC0A2F3BDC0A2F009538DCA1
:10229E000A2F009535DC8395EDCF24E438E08E01CE
:1022AE000E94B721002339F427E438E08E010E9402
:1022BE00B721002349F103E000936F0908891989BA
:1022CE002A893B89009370090EE211E00E94EF42C9
:1022DE000091700902DC06E511E00E94EF42BEDCBF
:1022EE00093519F0093709F039CD22E013E00EEF68
:1022FE000E9451420091700900939C0A21E030E047
:10230E00A9010E9493432ACD29E438E08E010E9450
:10231E00B721002309F44CC020E01FEC01E07ADB6A
:10232E0002E61EE00E94EF423CDB0DE51EE00E943D
:10233E00EF4204E610E0A2DB01E01FE00E94EF4254
:10234E0080E00EC000919B00102F17FF0FC086DC9F
:10235E00FE01EC53FF4F90E0E80FF91F00838395C9
:10236E008035A0F440E050E060E070E08A019B010F
:10237E00A801B9014F5F5F4F6F4F7F4F0030E0E014
:10238E001E07E4E02E07E0E03E07E0F20ADB20E065
:10239E0012E201E03FDB00E0FE01EC53FF4F90E064
:1023AE00E80FF91F00838E010C531F4F4ADCD6CC69
:1023BE0021E538E08E010E94B721002309F47AC08E
:1023CE00F89402E61EE00E94EF42EBDA0DE51EE005
:1023DE000E94EF4204E610E051DB00E91EE00E948D
:1023EE00EF4280E00EC000919B00102F17FF0FC030
:1023FE0035DCFE01EA5EFE4F90E0E80FF91F008328
:10240E0083958035A0F440E050E060E070E08A01F2
:10241E009B01A801B9014F5F5F4F6F4F7F4F003097
:10242E00E0E01E07E4E02E07E0E03E07E0F2B9DA56
:10243E0000E0FE01EA5EFE4F90E0E80FF91F008318
:10244E008E010A5E1E4FFDDB20E001C023952A306F
:10245E0090F4FE01EA5EFE4F30E0E20FF31F0081C2
:10246E000033A0F3FE01EA5EFE4F30E0E20FF31FF1
:10247E000081073458F780E010C0FE01EA5EFE4F7F
:10248E0030E0E20FF31F0081682F70E0605C7F4F39
:10249E00AB010E949343239583958C3070F304EF28
:1024AE0011E0ECDA789401E125E030E0A9010E9418
:1024BE00934354CC27E538E08E010E94B7210023C8
:1024CE0039F42AE538E08E010E94B721002391F0FD
:1024DE000DE91EE00E94EF4280E08C3008F03ECC09
:1024EE00282F30E0205C3F4FA9010E9487430CDB70
:1024FE008395F3CF24E638E08E010E94B7210023A6
:10250E0039F429E638E08E010E94B7210023B1F09C
:10251E0000E000936F090AE30093700922E012E0D5
:10252E0000919C0A0E945142002309F417CC00919D
:10253E009C0A0E3F09F412CCD9D510CC2BE638E00C
:10254E008E010E94B7210023C1F103E0801629F00D
:10255E0008E31FE00E94EF4201CCF8948888998826
:10256E00AA88BB884C885D886E887F880BE11FE047
:10257E000E94EF4216DA80E090E0A0E0B0E012C0D8
:10258E008C019D01080D191D2A1D3B1DF801322FCE
:10259E003BBF069000E00BBF002DB6DA8F5F9F4F5A
:1025AE00AF4FBF4F84159505A605B70548F3F9D96A
:1025BE0008EE13E063DA7894D1CB2FE737E08E0183
:1025CE000E94B7210023A9F103E0801629F008E349
:1025DE001FE00E94EF42C2CBF89488889988AA889F
:1025EE00BB884C885D886E887F880BE11FE00E9457
:1025FE00EF42D7D980E090E0A0E0B0E00FC08C01B0
:10260E009D01080D191D2A1D3B1D9801A9010E944F
:10261E0087437ADA8F5F9F4FAF4FBF4F8415950573
:10262E00A605B70560F3BDD908EE13E027DA789456
:10263E0095CB26E837E08E010E94B721002309F4DE
:10264E004DC003E0801629F008E31FE00E94EF4220
:10265E0085CBF89488889988AA88BB884C885D8831
:10266E006E887F8880E090E0A0E0B0E00DC0F6DAE2
:10267E00202FFE01E859FE4F8C01E00FF11F208341
:10268E008F5F9F4FAF4FBF4F84159505A605B705BA
:10269E0070F380E090E0A0E0B0E015C0FE01E859D4
:1026AE00FE4F8C01E00FF11F0081AC01BD01480D02
:1026BE00591D6A1D7B1D9A01A9010E9493438F5FCC
:1026CE009F4FAF4FBF4F84159505A605B70530F345
:1026DE0068D908EE13E0D2D9789440CB2DE837E0D4
:1026EE008E010E94B721002309F420C103E0801659
:1026FE0051F4488859886A887B880C891D892E89EF
:10270E003F89A02E0DC002E0801631F4488859880A
:10271E006A887B88A42C04C00FEE1DE00E94EF4255
:10272E0002E0801621F003E0801609F017CB00E0DE
:10273E000093A90A0093AA0A22E214E00EEFBDDA72
:10274E0002E209B90E94FE3B05C00BE611E00E94B1
:10275E00EF424394A41408F4DBC05524F201E25571
:10276E00F54F00810023A9F305E11EE00E94EF4220
:10277E00042DB3D990E09923B1F491E080E0873134
:10278E00D0F7082F10E0F801E255F54F0081002335
:10279E0041F020E011E0082F0E945142002309F47D
:1027AE0090E08395ECCF0CE11EE00E94EF4280E0BA
:1027BE000FC0841561F090E0FC01E255F54F0081E9
:1027CE00002329F025E01DE2082F0E946721839542
:1027DE00873178F306E21EE00E94EF422FEF1AEFE8
:1027EE00042D0E9467212EEF1DE2042D0E94672109
:1027FE00002309F4AACF04E610E040D90DE051D928
:10280E0000E00E9421210CE44CD900E00E9421211D
:10281E001A9A80E090ECA0E0B0E05524662477246C
:10282E0012C0FC013A2F3BBF069000E00BBF8F5F3A
:10283E009F4FAF4FBF4F500C002D62D95E9A01E0F3
:10284E00600E00E0701E0FEF601607E1700648F391
:10285E00052D56D95E9A5E9BFECF1A9800E00E9417
:10286E00212106E51ED900E00E94212100E001C0D1
:10287E000395043638F410E0F801ED52F64F10814E
:10288E001D32B1F70395202F01C00395043638F49D
:10289E0010E0F801ED52F64F10811D32B1F703959D
:1028AE0010E001C01395183090F4602F062F039599
:1028BE00422F242F239570E0FB01ED52F64F30810D
:1028CE0050E0FA01ED52F64F4081341759F31830AB
:1028DE00D1F401E31EE00E94EF4201E4E2D800E0F1
:1028EE000E94212107E4DDD800E00E94212120E092
:1028FE0017E0042D0E9451420CE211E0BFD800E017
:10290E000093A90A26CF0BE31EE00E94EF4221CFCF
:10291E000E94B84209B100939B0A20E030E0A90161
:10292E000E94934301E00093AA0A18CA24E937E0F3
:10293E008E010E94B721002309F444C000E00093E9
:10294E00AA0A0093A90A80E001E0801611F4AEEF06
:10295E0005C0088919892A893B89A02F0CE810E047
:10296E000E94EF4290E005C00DE2CED80DE5CCD826
:10297E0093959A17A8F40BE5C7D800E3C5D808E7D6
:10298E00C3D8092FAAD80AE3BFD820E011E0092F37
:10299E000E945142002341F30FE4B6D88395E6CF4F
:1029AE000DE0B2D80AE0B0D800E2AED8082FB4D805
:1029BE0004E512E00E94EF4201E00093AA0A0093A0
:1029CE00A90ACCC929E937E08E010E94B72100235C
:1029DE0009F457C001E0801619F4A0919C0A05C0B5
:1029EE00088919892A893B89A02F00E00093AA0A39
:1029FE000093A90A0DE911E00E94EF4280E001E484
:102A0E0012E00E94EF420A2F68D800919B00102F0F
:102A1E0017FF12C023D9802F823411F0823609F4A9
:102A2E00AA958E3411F08E3609F4A39507E612E0BE
:102A3E000E94EF420A2F51D809E100936F0901E07D
:102A4E000093700922E013E00A2F0E94514204E61F
:102A5E0010E014D809E100936F0900E000937009AB
:102A6E0022E013E00A2F0E94514204E610E00E9479
:102A7E00450D813511F0813741F601E00093AA0A28
:102A8E006DC92DE937E08E010E94B721002309F4AC
:102A9E0066C000E00093AA0A0AE036D880E02FC094
:102AAE00B0E0FD01ED52F64F00810F3F11F50A2FF8
:102ABE0010E00F5F1F4FF801ED52F64F00810F3FF0
:102ACE00C1F40AE712E00E94EF42082F0E94740D33
:102ADE0002E912E00E94EF420A2F10E00E5F1F4F34
:102AEE00F801ED52F64F00810E94740D0AE00E942B
:102AFE008B0DA3950091AB0AA01790F283958E3F94
:102B0E0008F589B920E011E00EEF0E94D5410DE0E5
:102B1E000E948B0D80FB26F40BE20E948B0D03C0EE
:102B2E000AE20E948B0D0FEF10E00E94450D0FEF91
:102B3E000E9435410093AB0A0091AB0A0023F1F2DB
:102B4E00A0E0D8CF00919B0A09B901E00093AA0A30
:102B5E000DE00E948B0D00E20E948B0DFFC824EA4F
:102B6E0037E08E010E94B721002399F104E0009313
:102B7E006F09088919892A893B890093700922E017
:102B8E0013E00EEF0E9451420AE912E00E94EF425A
:102B9E0000E814E82EE130E0488959896A897B897A
:102BAE004F5F5F4F6F4F7F4F0E940A440E94B20DDE
:102BBE0006EB12E00E94EF42088919892A893B89A7
:102BCE0009B900939B0A20E030E0A9010E949343CB
:102BDE00C5C829EA37E08E010E94B721002309F407
:102BEE0046C001E0801631F400E1402E55246624E3
:102BFE00772404C0488859886A887B880AEB11E0DC
:102C0E000E94EF422FC00091A80A1091A70A011747
:102C1E00B1F080E090E0A0E0B0E099240091A80A25
:102C2E0010E0F801E159F74F0081E8EAFAE010816F
:102C3E00139510830E94740D00E20E948B0D8F5F1E
:102C4E009F4FAF4FBF4F84159505A605B705D8F218
:102C5E00992041F40DE00E948B0D0AE00E948B0D2D
:102C6E009924939480E090E0A0E0B0E0ECCF21EBCB
:102C7E0037E08E010E94B721002309F461C0088954
:102C8E0019892A893B89A02F4C885D886E887F8898
:102C9E000AEB12E00E94EF420A2F0E94740D08EC1C
:102CAE0012E00E94EF4282010E940B0E02ED12E032
:102CBE000E94EF4280E00CC008E100936F0901E032
:102CCE000093700922E013E0082F0E945142839571
:102CDE00A81790F703EE12E00E94EF4214C00EE127
:102CEE0000936F090FEF0093700903E000937109D1
:102CFE0023E013E0082F0E9451428395A81778F71E
:102D0E0082010E94450D00919B00102F17FD26C8D1
:102D1E0080E00FC00EE100936F0900E00093700990
:102D2E0000E00093710923E013E0082F0E94514246
:102D3E008395A81778F782010E94450D80E0DECFBB
:102D4E0026EB37E08E010E94B721002309F4ECC078
:102D5E0000E00093AA0A00919C0A00936F0921E0FB
:102D6E0015E00EEF0E94514201E0801641F520E180
:102D7E0030E0A9010E948743802E80E090E0E82D8C
:102D8E00F0E031978E179F070CF042C0E82FF0E06D
:102D9E007196AF010E94874310E020E030E0FE0103
:102DAE007096482F50E0440F551F440F551FE40FE7
:102DBE00F51F00831183228333838395DFCF05E1D3
:102DCE00801610F004E1802E20E130E0082DA901DC
:102DDE000E94934380E015C0FE017096082F10E00C
:102DEE00000F111F000F111FE00FF11F0081118145
:102DFE0022813381E82FF0E07196AF010E94934358
:102E0E00839590E0E82DF0E031978E179F0724F31D
:102E1E000CE810E00E94EF420BE50E948B0D80E063
:102E2E0004C00DE50E948B0D839590E0E82DF0E037
:102E3E0031978E179F07DCF4FE017096082F10E075
:102E4E00000F111F000F111FE00FF11F00811181E4
:102E5E00228133810E94740D90E0E82DF0E03297CC
:102E6E008E179F07F4F60DE20E948B0DDDCF0091B9
:102E7E009B00102F17FD53C00CE810E00E94EF428C
:102E8E0080E019C0FE017096082F10E0000F111F90
:102E9E00000F111FE00FF11F00811181228133817C
:102EAE00102F00919C0A0E943D0E0E94740D00E2AC
:102EBE000E948B0D839590E0E82DF0E031978E17F0
:102ECE009F07ACF605E019E1FE017096282F30E061
:102EDE00220F331F220F331FE20FF31F4081518148
:102EEE006281738150E0040F151FF80104910230C6
:102EFE0049F6FE017096082F10E0000F111F000F0B
:102F0E00111FE00FF11F0081118122813381102FDB
:102F1E0000919C0A0E944D0E0E940B0EC8CF01E03C
:102F2E000093AA0A0C94B50E2AEB37E08E010E948C
:102F3E00B721002309F447C0488859886A887B88DE
:102F4E008C899D89AE89BF8900E00093AA0AA0E012
:102F5E004A1608F108E100936F0901E00093700929
:102F6E0022E013E00A2F0E945142A395F1CF0EE109
:102F7E0000936F090FEF0093700903E0009371093E
:102F8E0023E013E00A2F0E945142A3954A1678F7C8
:102F9E008C010E94450DA0E00FC00EE100936F0959
:102FAE0000E00093700900E00093710923E013E044
:102FBE000A2F0E945142A3954A1678F78C010E945F
:102FCE00450DA0E0E3CF2FEB37E08E010E94B72135
:102FDE00002369F0088919892A893B8900939C0A84
:102FEE0021E030E0A9010E9493430C94B50E27EF27
:102FFE0037E08E010E94B721002339F425EF37E028
:10300E008E010E94B721002321F00E9407410C94EB
:10301E00B50E20EF37E08E010E94B721002319F084
:10302E001CD00C94B50E2BEE37E08E010E94B7210A
:10303E00002321F0CC24C3940C94B50E0CED17E0B4
:10304E000E94280E0C94B50E00E00093AA0AEF968B
:10305E00E396DE5FEDE00C94674402E419E00E9413
:10306E00EF4205E619E00E94EF420CE819E00E94DB
:10307E00EF4202EB19E00E94EF420CEF19E00E94C2
:10308E00EF4204E41AE00E94EF420CE71AE00E94BD
:10309E00EF4203EA1AE00E94EF420FED1AE00E949F
:1030AE00EF420EE11BE00E94EF420BE31BE00E9499
:1030BE00EF4206E61BE00E94EF4202EA1BE00E948E
:1030CE00EF4208EE1BE00E94EF4202E31CE00E947A
:1030DE00EF4207E71CE00E94EF4205EB1CE00E9466
:1030EE00EF4203E01DE00E94EF4208950E9461440A
:1030FE0080E007E113E00E94EF42082F0E94930D3B
:10310E0001E11EE00E94EF42082F0E94740D0DE0B7
:10311E001EE00E94EF42A82FB0E01596FD01ED5281
:10312E00F64F00810E94930D01E11EE00E94EF42D6
:10313E00A82FB0E01596FD01ED52F64F00810E94CA
:10314E00740D09E20E948B0D839506E413E00E9434
:10315E00EF42082F0E94930D01E11EE00E94EF4204
:10316E00082F0E94740D0DE01EE00E94EF42A82F62
:10317E00B0E01596FD01ED52F64F00810E94930DC1
:10318E0001E11EE00E94EF42A82FB0E01596FD016E
:10319E00ED52F64F00810E94740D09E20E948B0DD4
:1031AE00839505E613E00E94EF42082F0E94930DCF
:1031BE0001E11EE00E94EF42082F0E94740D0DE007
:1031CE001EE00E94EF42A82FB0E01596FD01ED52D1
:1031DE00F64F00810E94930D01E11EE00E94EF4226
:1031EE00A82FB0E01596FD01ED52F64F00810E941A
:1031FE00740D09E20E948B0D839504E813E00E9482
:10320E00EF42082F0E94930D01E11EE00E94EF4253
:10321E00082F0E94740D0DE01EE00E94EF42A82FB1
:10322E00B0E01596FD01ED52F64F00810E94930D10
:10323E0001E11EE00E94EF42A82FB0E01596FD01BD
:10324E00ED52F64F00810E94740D09E20E948B0D23
:10325E00839503EA13E00E94EF42082F0E94930D1C
:10326E0001E11EE00E94EF42082F0E94740D0DE056
:10327E001EE00E94EF42A82FB0E01596FD01ED5220
:10328E00F64F00810E94930D01E11EE00E94EF4275
:10329E00A82FB0E01596FD01ED52F64F00810E9469
:1032AE00740D09E20E948B0D839502EC13E00E94CF
:1032BE00EF42082F0E94930D01E11EE00E94EF42A3
:1032CE00082F0E94740D0DE01EE00E94EF42A82F01
:1032DE00B0E01596FD01ED52F64F00810E94930D60
:1032EE0001E11EE00E94EF42A82FB0E01596FD010D
:1032FE00ED52F64F00810E94740D09E20E948B0D73
:10330E00839501EE13E00E94EF42082F0E94930D69
:10331E0001E11EE00E94EF42082F0E94740D0DE0A5
:10332E001EE00E94EF42A82FB0E01596FD01ED526F
:10333E00F64F00810E94930D01E11EE00E94EF42C4
:10334E00A82FB0E01596FD01ED52F64F00810E94B8
:10335E00740D09E20E948B0D839500E014E00E942B
:10336E00EF42082F0E94930D01E11EE00E94EF42F2
:10337E00082F0E94740D0DE01EE00E94EF42A82F50
:10338E00B0E01596FD01ED52F64F00810E94930DAF
:10339E0001E11EE00E94EF42A82FB0E01596FD015C
:1033AE00ED52F64F00810E94740D09E20E948B0DC2
:1033BE0083950FE114E00E94EF42082F0E94930DB7
:1033CE0001E11EE00E94EF42082F0E94740D0DE0F5
:1033DE001EE00E94EF42A82FB0E01596FD01ED52BF
:1033EE00F64F00810E94930D01E11EE00E94EF4214
:1033FE00A82FB0E01596FD01ED52F64F00810E9408
:10340E00740D09E20E948B0D83950EE314E00E9469
:10341E00EF42082F0E94930D01E11EE00E94EF4241
:10342E00082F0E94740D0DE01EE00E94EF42A82F9F
:10343E00B0E01596FD01ED52F64F00810E94930DFE
:10344E0001E11EE00E94EF42A82FB0E01596FD01AB
:10345E00ED52F64F00810E94740D09E20E948B0D11
:10346E0083950DE514E00E94EF42082F0E94930D04
:10347E0001E11EE00E94EF42082F0E94740D0DE044
:10348E001EE00E94EF42A82FB0E01596FD01ED520E
:10349E00F64F00810E94930D01E11EE00E94EF4263
:1034AE00A82FB0E01596FD01ED52F64F00810E9457
:1034BE00740D09E20E948B0D83950CE714E00E94B7
:1034CE00EF42082F0E94930D01E11EE00E94EF4291
:1034DE00082F0E94740D0DE01EE00E94EF42A82FEF
:1034EE00B0E01596FD01ED52F64F00810E94930D4E
:1034FE0001E11EE00E94EF42A82FB0E01596FD01FB
:10350E00ED52F64F00810E94740D09E20E948B0D60
:10351E0083950BE914E00E94EF42082F0E94930D51
:10352E0001E11EE00E94EF42082F0E94740D0DE093
:10353E001EE00E94EF42A82FB0E01596FD01ED525D
:10354E00F64F00810E94930D01E11EE00E94EF42B2
:10355E00A82FB0E01596FD01ED52F64F00810E94A6
:10356E00740D09E20E948B0D83950AEB14E00E9404
:10357E00EF42082F0E94930D01E11EE00E94EF42E0
:10358E00082F0E94740D0DE01EE00E94EF42A82F3E
:10359E00B0E01596FD01ED52F64F00810E94930D9D
:1035AE0001E11EE00E94EF42A82FB0E01596FD014A
:1035BE00ED52F64F00810E94740D09E20E948B0DB0
:1035CE00839509ED14E00E94EF42082F0E94930D9F
:1035DE0001E11EE00E94EF42082F0E94740D0DE0E3
:1035EE001EE00E94EF42A82FB0E01596FD01ED52AD
:1035FE00F64F00810E94930D01E11EE00E94EF4202
:10360E00A82FB0E01596FD01ED52F64F00810E94F5
:10361E00740D09E20E948B0D839508EF14E00E9451
:10362E00EF42082F0E94930D01E11EE00E94EF422F
:10363E00082F0E94740D0DE01EE00E94EF42A82F8D
:10364E00B0E01596FD01ED52F64F00810E94930DEC
:10365E0001E11EE00E94EF42A82FB0E01596FD0199
:10366E00ED52F64F00810E94740D09E20E948B0DFF
:10367E00839507E115E00E94EF42082F0E94930DFB
:10368E0001E11EE00E94EF42082F0E94740D0DE032
:10369E001EE00E94EF42A82FB0E01596FD01ED52FC
:1036AE00F64F00810E94930D01E11EE00E94EF4251
:1036BE00A82FB0E01596FD01ED52F64F00810E9445
:1036CE00740D09E20E948B0D839506E315E00E94AE
:1036DE00EF42082F0E94930D01E11EE00E94EF427F
:1036EE00082F0E94740D0DE01EE00E94EF42A82FDD
:1036FE00B0E01596FD01ED52F64F00810E94930D3C
:10370E0001E11EE00E94EF42A82FB0E01596FD01E8
:10371E00ED52F64F00810E94740D09E20E948B0D4E
:10372E00839505E515E00E94EF42082F0E94930D48
:10373E0001E11EE00E94EF42082F0E94740D0DE081
:10374E001EE00E94EF42A82FB0E01596FD01ED524B
:10375E00F64F00810E94930D01E11EE00E94EF42A0
:10376E00A82FB0E01596FD01ED52F64F00810E9494
:10377E00740D09E20E948B0D839504E715E00E94FB
:10378E00EF42082F0E94930D01E11EE00E94EF42CE
:10379E00082F0E94740D0DE01EE00E94EF42A82F2C
:1037AE00B0E01596FD01ED52F64F00810E94930D8B
:1037BE0001E11EE00E94EF42A82FB0E01596FD0138
:1037CE00ED52F64F00810E94740D09E20E948B0D9E
:1037DE00839503E915E00E94EF42082F0E94930D96
:1037EE0001E11EE00E94EF42082F0E94740D0DE0D1
:1037FE001EE00E94EF42A82FB0E01596FD01ED529B
:10380E00F64F00810E94930D01E11EE00E94EF42EF
:10381E00A82FB0E01596FD01ED52F64F00810E94E3
:10382E00740D09E20E948B0D839502EB15E00E9448
:10383E00EF42082F0E94930D01E11EE00E94EF421D
:10384E00082F0E94740D0DE01EE00E94EF42A82F7B
:10385E00B0E01596FD01ED52F64F00810E94930DDA
:10386E0001E11EE00E94EF42A82FB0E01596FD0187
:10387E00ED52F64F00810E94740D09E20E948B0DED
:10388E00839501ED15E00E94EF42082F0E94930DE3
:10389E0001E11EE00E94EF42082F0E94740D0DE020
:1038AE001EE00E94EF42A82FB0E01596FD01ED52EA
:1038BE00F64F00810E94930D01E11EE00E94EF423F
:1038CE00A82FB0E01596FD01ED52F64F00810E9433
:1038DE00740D09E20E948B0D839500EF15E00E9496
:1038EE00EF42082F0E94930D01E11EE00E94EF426D
:1038FE00082F0E94740D0DE01EE00E94EF42A82FCB
:10390E00B0E01596FD01ED52F64F00810E94930D29
:10391E0001E11EE00E94EF42A82FB0E01596FD01D6
:10392E00ED52F64F00810E94740D09E20E948B0D3C
:10393E0083950DEF12E00E94EF420E94350E0FE0CC
:10394E0016E00E94EF42082F0E94930D01E11EE047
:10395E000E94EF42082F0E94740D0DE01EE00E949F
:10396E00EF42A82FB0E01596FD01ED52F64F008103
:10397E000E94930D01E11EE00E94EF42A82FB0E0DD
:10398E001596FD01ED52F64F00810E94740D09E26D
:10399E000E948B0D83950BE316E00E94EF42082FD9
:1039AE000E94930D01E11EE00E94EF42082F0E943B
:1039BE00740D0DE01EE00E94EF42A82FB0E01596A8
:1039CE00FD01ED52F64F00810E94930D01E11EE0C4
:1039DE000E94EF42A82FB0E01596FD01ED52F64F72
:1039EE0000810E94740D09E20E948B0D83950AE5F9
:1039FE0016E00E94EF42082F0E94930D01E11EE097
:103A0E000E94EF42082F0E94740D0DE01EE00E94EE
:103A1E00EF42A82FB0E01596FD01ED52F64F008152
:103A2E000E94930D01E11EE00E94EF42A82FB0E02C
:103A3E001596FD01ED52F64F00810E94740D09E2BC
:103A4E000E948B0D839509E716E00E94EF42082F26
:103A5E000E94930D01E11EE00E94EF42082F0E948A
:103A6E00740D0DE01EE00E94EF42A82FB0E01596F7
:103A7E00FD01ED52F64F00810E94930D01E11EE013
:103A8E000E94EF42A82FB0E01596FD01ED52F64FC1
:103A9E0000810E94740D09E20E948B0D839508E946
:103AAE0016E00E94EF42082F0E94930D01E11EE0E6
:103ABE000E94EF42082F0E94740D0DE01EE00E943E
:103ACE00EF42A82FB0E01596FD01ED52F64F0081A2
:103ADE000E94930D01E11EE00E94EF42A82FB0E07C
:103AEE001596FD01ED52F64F00810E94740D09E20C
:103AFE000E948B0D839507EB16E00E94EF42082F74
:103B0E000E94930D01E11EE00E94EF42082F0E94D9
:103B1E00740D0DE01EE00E94EF42A82FB0E0159646
:103B2E00FD01ED52F64F00810E94930D01E11EE062
:103B3E000E94EF42A82FB0E01596FD01ED52F64F10
:103B4E0000810E94740D09E20E948B0D839506ED93
:103B5E0016E00E94EF42082F0E94930D01E11EE035
:103B6E000E94EF42082F0E94740D0DE01EE00E948D
:103B7E00EF42A82FB0E01596FD01ED52F64F0081F1
:103B8E000E94930D01E11EE00E94EF42A82FB0E0CB
:103B9E001596FD01ED52F64F00810E94740D09E25B
:103BAE000E948B0D839505EF16E00E94EF42082FC1
:103BBE000E94930D01E11EE00E94EF42082F0E9429
:103BCE00740D0DE01EE00E94EF42A82FB0E0159696
:103BDE00FD01ED52F64F00810E94930D01E11EE0B2
:103BEE000E94EF42A82FB0E01596FD01ED52F64F60
:103BFE0000810E94740D09E20E948B0D839504E1F1
:103C0E0017E00E94EF42082F0E94930D01E11EE083
:103C1E000E94EF42082F0E94740D0DE01EE00E94DC
:103C2E00EF42A82FB0E01596FD01ED52F64F008140
:103C3E000E94930D01E11EE00E94EF42A82FB0E01A
:103C4E001596FD01ED52F64F00810E94740D09E2AA
:103C5E000E948B0D839503E317E00E94EF42082F1D
:103C6E000E94930D01E11EE00E94EF42082F0E9478
:103C7E00740D0DE01EE00E94EF42A82FB0E01596E5
:103C8E00FD01ED52F64F00810E94930D01E11EE001
:103C9E000E94EF42A82FB0E01596FD01ED52F64FAF
:103CAE0000810E94740D09E20E948B0D839502E53E
:103CBE0017E00E94EF42082F0E94930D01E11EE0D3
:103CCE000E94EF42082F0E94740D0DE01EE00E942C
:103CDE00EF42A82FB0E01596FD01ED52F64F008190
:103CEE000E94930D01E11EE00E94EF42A82FB0E06A
:103CFE001596FD01ED52F64F00810E94740D09E2FA
:103D0E000E948B0D839501E717E00E94EF42082F6A
:103D1E000E94930D01E11EE00E94EF42082F0E94C7
:103D2E00740D0DE01EE00E94EF42A82FB0E0159634
:103D3E00FD01ED52F64F00810E94930D01E11EE050
:103D4E000E94EF42A82FB0E01596FD01ED52F64FFE
:103D5E0000810E94740D09E20E948B0D839500E98B
:103D6E0017E00E94EF42082F0E94930D01E11EE022
:103D7E000E94EF42082F0E94740D0DE01EE00E947B
:103D8E00EF42A82FB0E01596FD01ED52F64F0081DF
:103D9E000E94930D01E11EE00E94EF42A82FB0E0B9
:103DAE001596FD01ED52F64F00810E94740D09E249
:103DBE000E948B0D83950FEA17E00E94EF42082FA9
:103DCE000E94930D01E11EE00E94EF42082F0E9417
:103DDE00740D0DE01EE00E94EF42A82FB0E0159684
:103DEE00FD01ED52F64F00810E94930D01E11EE0A0
:103DFE000E94EF42A82FB0E01596FD01ED52F64F4E
:103E0E0000810E94740D09E20E948B0D83950EECC9
:103E1E0017E00E94EF42082F0E94930D01E11EE071
:103E2E000E94EF42082F0E94740D0DE01EE00E94CA
:103E3E00EF42A82FB0E01596FD01ED52F64F00812E
:103E4E000E94930D01E11EE00E94EF42A82FB0E008
:103E5E001596FD01ED52F64F00810E94740D09E298
:103E6E000E948B0D83950DEE17E00E94EF42082FF6
:103E7E000E94930D01E11EE00E94EF42082F0E9466
:103E8E00740D0DE01EE00E94EF42A82FB0E01596D3
:103E9E00FD01ED52F64F00810E94930D01E11EE0EF
:103EAE000E94EF42A82FB0E01596FD01ED52F64F9D
:103EBE0000810E94740D09E20E948B0D83950CE027
:103ECE0018E00E94EF42082F0E94930D01E11EE0C0
:103EDE000E94EF42082F0E94740D0DE01EE00E941A
:103EEE00EF42A82FB0E01596FD01ED52F64F00817E
:103EFE000E94930D01E11EE00E94EF42A82FB0E058
:103F0E001596FD01ED52F64F00810E94740D09E2E7
:103F1E000E948B0D83950BE218E00E94EF42082F52
:103F2E000E94930D01E11EE00E94EF42082F0E94B5
:103F3E00740D0DE01EE00E94EF42A82FB0E0159622
:103F4E00FD01ED52F64F00810E94930D01E11EE03E
:103F5E000E94EF42A82FB0E01596FD01ED52F64FEC
:103F6E0000810E94740D09E20E948B0D83950AE474
:103F7E0018E00E94EF42082F0E94930D01E11EE00F
:103F8E000E94EF42082F0E94740D0DE01EE00E9469
:103F9E00EF42A82FB0E01596FD01ED52F64F0081CD
:103FAE000E94930D01E11EE00E94EF42A82FB0E0A7
:103FBE001596FD01ED52F64F00810E94740D09E237
:103FCE000E948B0D839509E618E00E94EF42082FA0
:103FDE000E94930D01E11EE00E94EF42082F0E9405
:103FEE00740D0DE01EE00E94EF42A82FB0E0159672
:103FFE00FD01ED52F64F00810E94930D01E11EE08E
:10400E000E94EF42A82FB0E01596FD01ED52F64F3B
:10401E0000810E94740D09E20E948B0D839508E8C1
:10402E0018E00E94EF42082F0E94930D01E11EE05E
:10403E000E94EF42082F0E94740D0DE01EE00E94B8
:10404E00EF42A82FB0E01596FD01ED52F64F00811C
:10405E000E94930D01E11EE00E94EF42A82FB0E0F6
:10406E001596FD01ED52F64F00810E94740D09E286
:10407E000E948B0D839507EA18E00E94EF42082FED
:10408E000E94930D01E11EE00E94EF42082F0E9454
:10409E00740D0DE01EE00E94EF42A82FB0E01596C1
:1040AE00FD01ED52F64F00810E94930D01E11EE0DD
:1040BE000E94EF42A82FB0E01596FD01ED52F64F8B
:1040CE0000810E94740D09E20E948B0D839506EC0F
:1040DE0018E00E94EF42082F0E94930D01E11EE0AE
:1040EE000E94EF42082F0E94740D0DE01EE00E9408
:1040FE00EF42A82FB0E01596FD01ED52F64F00816C
:10410E000E94930D01E11EE00E94EF42A82FB0E045
:10411E001596FD01ED52F64F00810E94740D09E2D5
:10412E000E948B0D839505EE18E00E94EF42082F3A
:10413E000E94930D01E11EE00E94EF42082F0E94A3
:10414E00740D0DE01EE00E94EF42A82FB0E0159610
:10415E00FD01ED52F64F00810E94930D01E11EE02C
:10416E000E94EF42A82FB0E01596FD01ED52F64FDA
:10417E0000810E94740D09E20E948B0D839504E06C
:10418E0019E00E94EF42082F0E94930D01E11EE0FC
:10419E000E94EF42082F0E94740D0DE01EE00E9457
:1041AE00EF42A82FB0E01596FD01ED52F64F0081BB
:1041BE000E94930D01E11EE00E94EF42A82FB0E095
:1041CE001596FD01ED52F64F00810E94740D09E225
:1041DE000E948B0D839503E219E00E94EF42082F97
:1041EE000E94930D01E11EE00E94EF42082F0E94F3
:1041FE00740D0DE01EE00E94EF42A82FB0E0159660
:10420E00FD01ED52F64F00810E94930D01E11EE07B
:10421E000E94EF42A82FB0E01596FD01ED52F64F29
:10422E0000810E94740D09E20E948B0D8395E4E0DB
:10423E000C9470449A938A93902F80E00091A80A70
:10424E001091A70A0117D1F340E050E060E070E052
:10425E000091A80A1091A70A0117A1F48A019B01E7
:10426E00A801B9014F5F5F4F6F4F7F4F013EE3E9EA
:10427E001E07E4E02E07E0E03E0750F3082F899179
:10428E00999108950091A80A10E0F801E159F74FAD
:10429E000081E8EAFAE0108113951083282F30E0B0
:1042AE00F901ED52F64F0083992341F0082F10E0EB
:1042BE00F801ED52F64F00810E948B0D8395C4CF0D
:1042CE000E946144902FA12FB22FA0936F09B0933B
:1042DE00700900EF0093710905E5009372090FE074
:1042EE00009373090AEA0093740926E01DE0092F72
:1042FE000E94D541802F0091AA0A002349F00CE8B4
:10430E0010E00E94EF42282F07E31AE00E94244299
:10431E000AE010E00E94450D1A2F092F0E943D0E53
:10432E000B1711F401E001C000E0E4E00C947044BE
:10433E00A80100E001C00395083C88F410E0F901E3
:10434E00E00FF11F608110E0FA01E00FF11F6083B2
:10435E0010E0F901E00FF11F1081112361F70895AC
:10436E00A80100E010E0FA01E00FF11F608110E0FB
:10437E00F901E00FF11F1081611791F4039510E020
:10438E00FA01E00FF11F1081112339F410E0F90149
:10439E00E00FF11F1081112321F0093C18F308954D
:1043AE0000E008950E945D440901BA0180E001C059
:1043BE00839590E0FB01E80FF91F20812032C1F3B5
:1043CE008C3360F590E0FB01E80FF91F208122236A
:1043DE0029F120E00DC090E0FB01E80FF91F4081AC
:1043EE004F7530E0F801E20FF31F4083239583955C
:1043FE0090E0FB01E80FF91F3081303348F090E078
:10440E00FB01E80FF91F30813B3710F4803118F3B0
:10441E0040E030E0F801E20FF31F4083E02FF12F70
:10442E000081002311F400E0B7C0A0E0B0C0839576
:10443E0090E0FB01E80FF91F00810032C1F390E01C
:10444E00FB01E80FF91F0081002319F4A3950A2F31
:10445E00A3C000E010E020E030E04A2F50E0440F0F
:10446E00551F440F551FF001E40FF51F00831183F4
:10447E002283338356C090E0FB01E80FF91F0081C1
:10448E00013408F44DC090E0FB01E80FF91F0081E4
:10449E000B3708F045C090E0FB01E80FF91F0081D3
:1044AE000F7500830A2F10E0000F111F000F111F50
:1044BE00F001E00FF11F008111812281338144E070
:1044CE000E9402444A2F50E0440F551F440F551FBF
:1044DE00F001E40FF51F008311832283338390E0F4
:1044EE00FB01E80FF91F008110E007531040212F48
:1044FE00220F220B322F4A2F50E0440F551F440F2C
:10450E00551FF001E40FF51F4080518062807380CB
:10451E00400E511E621E731E408251826282738251
:10452E0083958C3398F590E0FB01E80FF91F00811D
:10453E00002319F4AE5F0A2F2FC090E0FB01E80FA5
:10454E00F91F00810B33E1F090E0FB01E80FF91F3A
:10455E0000810A33A9F090E0FB01E80FF91F0081FA
:10456E000C3271F090E0FB01E80FF91F00810E3262
:10457E0039F090E0FB01E80FF91F0081003279F469
:10458E0000E290E0FB01E80FF91F0083A395AE3126
:10459E0008F44ECFA3950A2FE8E00C946C4490E0FB
:1045AE00FB01E80FF91F0081003308F464CF90E09F
:1045BE00FB01E80FF91F00810A3308F05CCF0A2FC8
:1045CE0010E0000F111F000F111FF001E00FF11F7F
:1045DE00008111812281338144E00E9402444A2FDE
:1045EE0050E0440F551F440F551FF001E40FF51F07
:1045FE00008311832283338390E0FB01E80FF91FC0
:10460E00008110E000531040212F220F220B322F79
:10461E004A2F50E0440F551F440F551FF001E40F71
:10462E00F51F4080518062807380400E511E621EC5
:10463E00731E408251826282738272CF0E946144E5
:10464E00C801A22FB1E016C008E00E948B0D00E257
:10465E000E948B0D08E00E948B0D0A2FA02FAA95A9
:10466E00002391F72EE83EE08C0162DEA02F8C0134
:10467E000E94280EBB2309F446C000919B00102F08
:10468E0017FD0CC00D99F9CF2DED36E08C0150DEE3
:10469E00A02F8C010E94280E01E036C000919C00D4
:1046AE00102F105039F31A95C1F2175099F012507D
:1046BE0029F0135019F01E50E9F219C000E0B0E0D5
:1046CE00FC01EA0FFB1F00839C010EE81EE030DEAA
:1046DE0001E01AC0A13070F2AA9508E00E948B0D7D
:1046EE0000E20E948B0D08E00E948B0DC3CFAC330D
:1046FE0008F62A2F30E0FC01E20FF31F00830E9420
:10470E008B0DA395B7CF00E0E4E00C9470440E94AB
:10471E006144902F812F983050F5883040F5092F45
:10472E0010E00F5F1F4F40E450E00E94A543D801F8
:10473E00082F10E00F5F1F4F40E450E00E94A5438A
:10474E0020E011C0422F50E0400F511FFA01E35AF2
:10475E00F44F3081422F50E04A0F5B1FFA01E35AAB
:10476E00F44F30832395203468F3092F03D0E4E00F
:10477E000C9470449A938A93902F973011F490E092
:10478E0001C0939580E007C0182F092FEED1182F86
:10479E00092F27D183958731B8F317E1092FE5D17A
:1047AE0017E1092FCFD0F801E35AF44F00810E9490
:1047BE00740D18E1092FD9D118E1092FC3D0F801D2
:1047CE00E35AF44F00810E94740D899199910895D6
:1047DE00005049F00A9561F00A9579F00A9591F02A
:1047EE000A95A9F0089505E818E10E94EF42089590
:1047FE0009E918E10E94EF42089507EA18E10E94C4
:10480E00EF4208950AEB18E10E94EF4208950AEC78
:10481E0018E10E94EF4208959A938A93802F912F68
:10482E00EBEEF8E11491E2EEF8E104910E9493327E
:10483E00082F0E94740DECEEF8E11491E3EEF8E10E
:10484E0004910E949332092F0E94740DEDEEF8E14F
:10485E001491E4EEF8E104910E949332192F082F7F
:10486E0071D00E940B0E8991999108958A93E5EE6D
:10487E00F8E11491ECEDF8E104910E94933280E09E
:10488E0004C000E20E948B0D83958634D0F3E5EED2
:10489E00F8E11491ECEDF8E104910E9493328991C4
:1048AE0008959A938A939091710B80E00CC0182F03
:1048BE000091CA0E039559D108E00E948B0D00E2BB
:1048CE000E948B0D8395873190F380E00BC0182FDB
:1048DE00092F03954AD108E00E948B0D0CE70E9428
:1048EE008B0D8395873198F39093CA0EE9EEF8E11C
:1048FE001491E0EEF8E104910E949332092F0E9488
:10490E00740D899199910895093031F4133020F086
:10491E00143110F401E00895083021F4173110F429
:10492E0001E00895083030F4183111F0173111F408
:10493E0001E00895083020F4183110F402E00895D3
:10494E0000E00895682F202F812F222371F48731E4
:10495E0038F4082F10E0000F111F00501E4F39C001
:10496E00082F10E0095D1D4F34C0873149F4022F26
:10497E0010E040E450E00E94A543025C1F4F29C0A6
:10498E00883149F4022F10E040E450E00E94A54324
:10499E00015C1F4F1EC0283029F4082F10E0005E66
:1049AE001F4F17C0293029F4082F10E0055F1F4F45
:1049BE0010C0022F10E00150104040E450E00E9461
:1049CE00A543980102E0809F8001020F131F005C37
:1049DE001F4F003422E0120710F000E010E0862F87
:1049EE0008959A938A93902F812F873100F5182F6F
:1049FE00092FA8DFF801E35AF44F018107FF0DC01C
:104A0E000DE20E948B0D0DE20E948B0D0DE20E94B5
:104A1E008B0D0DE20E948B0D0AC0182F092F92DF0D
:104A2E00F801E35AF44F008111810E940B0E899117
:104A3E00999108950E9461440091630E002351F0F4
:104A4E0000E0C6DE0E94350E093521F0093711F05F
:104A5E0000E088C0E1E6FEE00081118120E030E058
:104A6E0040E052E060E070E00E94E643A801B90128
:104A7E00405050426F4F7F4F80E0A0E0B0E017C033
:104A8E008D0120E030E0040F151F261F371FF8019F
:104A9E00322F3BBF069000E00BBFFD01E35AF44FEF
:104AAE000082FD01E35AF44F0081800F1196A03071
:104ABE0002E0B00728F3A0E00DC020E030E802E0ED
:104ACE00A09F800100501E4FF801E35AF44F20833F
:104ADE003183A395A731B8F4B0E0FD01E255F54F4F
:104AEE000081002351F31EE10A2F0E94673222E05B
:104AFE00A29F20E0020E22E0121EF001E35AF44FB4
:104B0E0000831183E6CF8F3F21F40091710B0830A3
:104B1E00D8F0A0E0B0E006C000E0FD01E35AF44F8B
:104B2E0000831196A03002E0B007B0F300E00093CE
:104B3E00710B0FEF00936E0B00936B0B00E2009363
:104B4E00730B00E20093750B0091740B053018F097
:104B5E0000E00093740B00E000936A0B00E00093FA
:104B6E00630E01E0E4E00C9470449A938A9362978A
:104B7E00602F212FCE010896EFE9F9E830E08C0185
:104B8E004AE050E00E944644CE01E7E9F9E830E001
:104B9E008C0148E050E00E944644283111F0273144
:104BAE0051F42395122FFE0170E0E60FF71F0081DE
:104BBE000E94933210C0273158F42395122FFE0114
:104BCE00389670E0E60FF71F00810E94933203C003
:104BDE0001E20E948B0D62968991999108950E942F
:104BEE00624480E005C00CE810E00E94EF4283951D
:104BFE008C33C8F311E001E00E94933206E51FE00A
:104C0E000E94EF4206E91FE00E94EF4203EE1FE012
:104C1E000E94EF420AE210E10E94EF4209E710E122
:104C2E000E94EF4208EC10E10E94EF4207E111E111
:104C3E000E94EF4206E611E10E94EF4205EB11E100
:104C4E000E94EF4204E012E10E94EF4203E512E1FE
:104C5E000E94EF4202EA12E10E94EF4201EF12E1DE
:104C6E000E94EF4200E413E10E94EF420FE813E1CD
:104C7E000E94EF420EED13E10E94EF420DE214E1AD
:104C8E000E94EF420CE714E10E94EF420BEC14E19C
:104C9E000E94EF420AE115E10E94EF4209E615E19A
:104CAE000E94EF4208EB15E10E94EF4209E016E187
:104CBE000E94EF42E1E6FEE000811181012B69F4D2
:104CCE0007E417E10E94EF4206E917E10E94EF4266
:104CDE0007EE17E10E94EF420CC008E516E10E94B4
:104CEE00EF4207EA16E10E94EF4208EF16E10E943A
:104CFE00EF4206E318E10E94EF4280E001C0839587
:104D0E008931F8F490E006C0A23019F4182F092F5B
:104D1E0068DE9395933198F7182F092FF5DDA02FA4
:104D2E00AA23B9F3182F092F20DFA13069F7182F06
:104D3E00092F08DEF801E35AF44F00810E94740D2A
:104D4E00E8CFAFDDE6EEF8E11491EDEDF8E1049178
:104D5E000E9493320DE51BE00E94280EE7EEF8E16B
:104D6E001491EEEDF8E104910E949332E1E6FEE03B
:104D7E00008111810E940B0EE8EEF8E11491EFED27
:104D8E00F8E104910E949332E1E6FEE00081118188
:104D9E0020E030E040E052E060E070E00E94E64348
:104DAE00005010422F4F3F4F0E94170EE3E00C941D
:104DBE0071440E945944EF976297DA95BE0164528E
:104DCE007F4FEEE7F9E830E08B0149E150E00E94B9
:104DDE004644A0E08A2EAA2EBA2E24EF3FE0A90167
:104DEE000E948743053511F40C942B311A2F082D90
:104DFE0013DD1A2F082DB9DE9090710B00919B00D8
:104E0E00102F17FD02C00D99F9CF0D9902C08DE03C
:104E1E0002C080919C008B31D1F50E94350E802FFF
:104E2E008B3519F40E94350E802F843421F488209E
:104E3E0089F08A940FC0833411F483940BC08134AB
:104E4E0021F4AA2339F0AA9505C0823419F4A831A9
:104E5E0008F4A395FE01E452FF4FB0E0EA0FFB1FEA
:104E6E000081081538F4FE01E452FF4FB0E0EA0F5E
:104E7E00FB1F80808B1421F4AA1511F40C944A3276
:104E8E001A2F082DC9DCB82CAA2E0C944A32803267
:104E9E0009F044C01A2F082D37DD023011F00C94A2
:104EAE004A3280E090E81A2F082D4CDDF801E35AC3
:104EBE00F44F008111810827192700831183882060
:104ECE0029F58A2F02E0809F800100501E4FF801C5
:104EDE00E35AF44F018107FD16C090E0FC01E25544
:104EEE00F54F0081002379F014E2082F0E946732FB
:104EFE0022E0829F20E0020E22E0121EF001E35A11
:104F0E00F44F008311830A2F0E94983B1A2F082D0D
:104F1E0068DD01E00093630E0C944A328D3509F082
:104F2E004CC01A2F082D21DE1A2F082DEDDC013072
:104F3E00B9F41A2F082D06DDF801E35AF44F00815B
:104F4E00039500831A2F082DFDDCF801E35AF44F68
:104F5E0000810E94740D01E00093630E0C944A329E
:104F6E00023011F00C944A321A2F082DEBDCF801A6
:104F7E00E35AF44F008111810F7F13700F3F23E02E
:104F8E00120711F40C944A321A2F082DDBDCF801AB
:104F9E00E35AF44F008111810F5F1F4F008311837D
:104FAE001A2F082D1EDD882019F40A2F0E94983B17
:104FBE0001E00093630E0C944A328B3509F04AC01F
:104FCE001A2F082DD2DD1A2F082D9EDC0130B9F4D0
:104FDE001A2F082DB7DCF801E35AF44F00810A9519
:104FEE0000831A2F082DAEDCF801E35AF44F00812E
:104FFE000E94740D01E00093630E0C944A3202304D
:10500E0011F00C944A321A2F082D9CDCF801E35A49
:10501E00F44F008111810F7F1370012B11F40C944A
:10502E004A321A2F082D8EDCF801E35AF44F008114
:10503E00118101501040008311831A2F082DD1DCED
:10504E00882019F40A2F0E94983B01E00093630E0A
:10505E000C944A328D3709F049C01A2F082D54DCB2
:10506E000130B9F41A2F082D6DDCF801E35AF44F14
:10507E000081005F00831A2F082D64DCF801E35ACB
:10508E00F44F00810E94740D01E00093630E0C94A6
:10509E004A32023011F00C944A321A2F082D52DC8B
:1050AE00F801E35AF44F008111810F7F13700F3E08
:1050BE0023E0120710F00C944A321A2F082D42DC0E
:1050CE00F801E35AF44F00811181005F1F4F0083F6
:1050DE0011831A2F082D85DC882019F40A2F0E94BF
:1050EE00983B01E00093630E0C944A328B3709F023
:1050FE0048C01A2F082D08DC0130B9F41A2F082DDC
:10510E0021DCF801E35AF44F0081005100831A2F7D
:10511E00082D18DCF801E35AF44F00810E94740D3B
:10512E0001E00093630E0C944A32023011F00C949D
:10513E004A321A2F082D06DCF801E35AF44F80810B
:10514E0091818F7F93708031904010F40C944A328D
:10515E001A2F082DF7DBF801E35AF44F0081118165
:10516E0000511040008311831A2F082D3ADC88203D
:10517E0019F40A2F0E94983B01E00093630E0C94E1
:10518E004A328F3281F51A2F082DBEDB023011F014
:10519E000C944A321A2F082DD5DBF801E35AF44F3E
:1051AE000081118100701077003020E7120710F097
:1051BE000C944A321A2F082DC5DBF801E35AF44F2E
:1051CE00008111810050104F008311831A2F082D7A
:1051DE0008DC882019F40A2F0E94983B01E0009306
:1051EE00630E0C944A328E3271F51A2F082D8CDB19
:1051FE00023011F00C944A321A2F082DA3DBF8015D
:10520E00E35AF44F0081118100701077012B11F4D5
:10521E000C944A321A2F082D95DBF801E35AF44FFD
:10522E000081118100501041008311831A2F082D27
:10523E00D8DB882019F40A2F0E94983B01E00093D6
:10524E00630E0C944A3212DB803360F08B3750F4CD
:10525E00082F0E948B0D88A721E08E01085D1F4F3D
:10526E00EDD905C020E08E01085D1F4FE7D900E0A3
:10527E000883AE01485D5F4F9E012C593F4F8E0152
:10528E0091D8B02FBB2311F40C944A3226E137E0AB
:10529E008E0166D8002341F0A2DCA0E08A2E1A2FE0
:1052AE00082DBADA0C944A3229E137E08E0158D82B
:1052BE00002331F429EA37E08E0152D8002359F148
:1052CE00E5EEF8E11491ECEDF8E104910E949332D1
:1052DE0025E030E0A9010E948743013191F40DE9E8
:1052EE001EE00E94EF4290E00AC0292F30E0205CC1
:1052FE003F4FA9010E9487430E948B0D93959C30CE
:10530E00A0F30E94840E6BDCA0E08A2E1A2F082DCB
:10531E0083DA0C944A322DE137E08E0121D8002336
:10532E00B1F0B33021F002E053DA0C944A32FE01B0
:10533E00FF9605A116A127A130A5802EFE01FF968E
:10534E0001A512A523A534A5A02F0C944A3222E262
:10535E0037E08E0105D8002339F427E237E08E01BD
:10536E000E94B721002349F1E1E6FEE02081318160
:10537E002F3700E03007E8F4E1E6FEE0008111810E
:10538E000F5F1F4F0083118355DB002341F027DC95
:10539E00A0E08A2E1A2F082D3FDA0C944A32E1E64D
:1053AE00FEE00081118101501040008311830C94A6
:1053BE004A3201E00DDA0C944A3229E237E08E01CE
:1053CE000E94B721002339F420E337E08E010E94BA
:1053DE00B721002339F1E1E6FEE000811181012BB6
:1053EE00E9F0E1E6FEE000811181015010400083FA
:1053FE00118320DB002341F0F2DBA0E08A2E1A2F6E
:10540E00082D0ADA0C944A32E1E6FEE000811181A1
:10541E000F5F1F4F008311830C944A3201E0D8D9DD
:10542E000C944A3222E337E08E010E94B72100230A
:10543E0039F422E438E08E010E94B7210023A1F155
:10544E00B23021F002E0C4D90C944A32FE01FF962C
:10545E0005A116A127A130A5003840E0140740E0B1
:10546E00240740E03407E8F4E1E6FEE08081918114
:10547E00FE01FF9605A116A127A130A5E1E6FEE0EB
:10548E0000831183D7DA002339F0A9DBA0E08A2E3E
:10549E001A2F082DC1D9F7C7E1E6FEE0808391836C
:1054AE00F2C701E095D9EFC727E337E08E010E94DE
:1054BE00B7210023D1F1B23019F002E089D9E3C748
:1054CE00FE01FF9605A116A127A130A5003840E0E8
:1054DE00140740E0240740E0340720F5E1E6FEE043
:1054EE0080819181FE01FF9605A116A127A130A50D
:1054FE00E1E6FEE0008311839DDA002371F0E1E620
:10550E00FEE0808391836BDBA0E08A2E1A2F082D9C
:10551E0083D901E00093630EB6C7E1E6FEE0808317
:10552E009183B1C701E054D9AEC725ED37E08E01A6
:10553E000E94B721002339F421ED37E08E010E943D
:10554E00B721002369F00FEF2FEF3FE0A9010E9472
:10555E00934308E001BD04E610E00E94450D93C799
:10556E002CE337E08E010E94B721002311F10AE3EC
:10557E000E948B0D20E08E01085D1F4F5FD8002327
:10558E0061F000E00DAB9E01285D3F4F0DE51BE085
:10559E000E949F2101E00093630EE6EEF8E1149164
:1055AE00EDEDF8E10491B8D70DE51BE00E94280E51
:1055BE006AC721E437E08E010E94B721002309F467
:1055CE0083C0B130A9F580E0873108F05CC702E0F6
:1055DE00809F00E0000E02E0101EF001E35AF44F2F
:1055EE00018107FF23C090E0FC01E255F54F0081D9
:1055FE000023B1F021E018E1082F0E946D0E14E295
:10560E00082F5ED722E0829F20E0020E22E0121EBB
:10561E00F001E35AF44F00831183082F0E94983B48
:10562E00182F00E0A2DA182F00E0DBD98395CCCF3B
:10563E0090E0092F10E0EB2FF0E031970E171F07C7
:10564E000CF021C7FE01EC59FF4F092F10E0000F9F
:10565E00111F000F111FE00FF11F00811181228118
:10566E003381802F02E0809F00E0000E02E0101ECA
:10567E00F001E35AF44F018107FF24C0082F10E018
:10568E00F801E255F54F00810023B1F021E018E159
:10569E00082F0E946D0E14E2082F12D722E0829F6F
:1056AE0020E0020E22E0121EF001E35AF44F0083B6
:1056BE001183082F0E94983B182F00E056DA182FFE
:1056CE0000E08FD99395B5CF24E437E08E010E9488
:1056DE00B721002309F461C0B13021F580E0873194
:1056EE0008F0D1C690E0FC01E255F54F0081002391
:1056FE0029F020E018E1082F0E946D0E02E0809F35
:10570E0000E0000E02E0101EF001E35AF44F01819A
:10571E0000680183182F00E028DA182F00E061D905
:10572E008395DDCF90E0092F10E0EB2FF0E031975D
:10573E000E171F070CF0A7C6FE01EC59FF4F092FDD
:10574E0010E0000F111F000F111FE00FF11F00815D
:10575E00118122813381802F082F10E0F801E2554C
:10576E00F54F0081002329F020E018E1082F0E9458
:10577E006D0E02E0809F00E0000E02E0101EF001B0
:10578E00E35AF44F018100680183182F00E0EDD930
:10579E00182F00E026D99395C6CF28E437E08E0166
:1057AE000E94B721002339F42DE437E08E010E94C8
:1057BE00B7210023B9F0FE01FF9605A116A127A17E
:1057CE0030A5B23019F002E003D85DC6083020F0E3
:1057DE0004E00E94EF2357C60093710B01E0009383
:1057EE00630E51C62FE437E08E010E94B7210023CD
:1057FE0039F423E537E08E010E94B721002399F199
:10580E00B33021F002E00E94EF233DC6FE01FF9669
:10581E0005A116A127A130A5C801FE01FF9601A57D
:10582E0012A523A534A5902F983010F4883020F0BF
:10583E0004E00E94EF2327C60AE30E948B0D082F77
:10584E000E94740D0DE20E948B0D0EE30E948B0DD3
:10585E00092F0E94740D182F092F0E948E2301E02C
:10586E000093630E10C62DE037E08E010E94B72123
:10587E00002341F42CEF37E08E010E94B721002364
:10588E0009F488C0B33020F002E00E94EF23FBC57C
:10589E00B13019F40091710B06C0FE01FF9605A1FF
:1058AE0016A127A130A5073020F004E00E94EF23B7
:1058BE00EAC5E1E6FEE020813181232B41F410910F
:1058CE00710B133020F004E00E94EF23DCC5B230E0
:1058DE0039F417E00E948E2301E00093630E19C085
:1058EE00B130A1F40091710B073080F417E00091F4
:1058FE00710B0E948E23EDE5FBE004890395048B6A
:10590E000E94582401E00093630E03C004E00E943D
:10591E00EF23E1E6FEE000811181012B09F0B3C512
:10592E000091710B013029F00091710B023009F0DA
:10593E00AAC500E410E020E830E040EC50E080E042
:10594E001EC062E0869F020E131EF001E35AF44F52
:10595E002080318062E0869F000E111EF001E35A16
:10596E00F44F60817181261A370A62E0869F040E19
:10597E00151EF001E35AF44F208231828395873150
:10598E0000F30E943D2403E00E94EF2302E00E94F8
:10599E00C12379C528E537E08E010E94B721002387
:1059AE0039F429E638E08E010E94B7210023E9F18F
:1059BE00B23029F5FE01FF9605A116A127A130A54B
:1059CE00C801873020F004E00E94EF235CC50091EF
:1059DE00710B801770F4EDE5FBE004890A95048BDA
:1059EE000E94582406C0182F1395082F0E948E234C
:1059FE0083958630C0F301E00093630E44C5B13049
:105A0E0009F041C50091710B013058F0EDE5FBE056
:105A1E0004890A95048B0E94582401E00093630EBA
:105A2E0032C504E00E94EF232EC52FE537E08E012C
:105A3E000E94B721002339F427E438E08E010E943A
:105A4E00B721002381F1FE01FF9605A116A127A122
:105A5E0030A5802FB23021F002E00E94EF2313C553
:105A6E00873020F004E00E94EF230DC596E006C0BB
:105A7E00192F1A95092F0E948E239A958917C0F314
:105A8E0017E0082F0E948E230091710B801738F4B7
:105A9E00EDE5FBE004890395048B0E94582401E098
:105AAE000093630EF0C423E338E08E010E94B72109
:105ABE00002339F426E338E08E010E94B72100233B
:105ACE00D1F1FE01FF9605A116A127A130A5902FB9
:105ADE00B23021F002E00E94EF23D5C4973020F0BF
:105AEE0004E00E94EF23CFC489E50091710B90175B
:105AFE0030F000E00E94EF230E94350E802F893592
:105B0E0019F0893709F0BFC4EAEEF8E11491E1EE1D
:105B1E00F8E1049101D5092F0E94740D192F07E0A9
:105B2E000E948E2380E0873108F0ADC4082F0E94BA
:105B3E00983B8395F8CF26E637E08E010E94B72179
:105B4E00002341F42BE637E08E010E94B72100239B
:105B5E0009F470C0B13051F401E010E020E030E003
:105B6E00FE01FF9605A316A327A330A720E030E081
:105B7E0010E20EEF0E94760E80E019C090E0FC015C
:105B8E00E255F54F0081002389F01EE1082F0E9497
:105B9E004D0E0F7F137022E0829F20E0020E22E056
:105BAE00121EF001E35AF44F00831183839587315F
:105BBE0028F30EEF0093670E0093640EFE01FF961E
:105BCE0005A116A127A130A53CD50EC000919B00C2
:105BDE00102F17FF09C00FEF0093640E0FE41FE0A4
:105BEE000E94EF420E94350E0091680E002371F75D
:105BFE0008ED18E10E94EF4280E016C090E0FC0133
:105C0E00E255F54F0081002371F01EE1082F58D4A4
:105C1E0022E0829F20E0020E22E0121EF001E35AE3
:105C2E00F44F008311838395873140F307E00E9480
:105C3E00C12329C422E737E08E010E94B721002339
:105C4E0009F44DC0B23021F002E00E94EF231BC4D4
:105C5E001A2F082D0E94BC251A2F082D0E948B2466
:105C6E000130E9F4FE01FF9605A116A127A130A58A
:105C7E00802F1A2F082D0E94A924F801E35AF44F01
:105C8E0080831A2F082D0E94A924F801E35AF44F9D
:105C9E0000810E94740D01E00093630EF4C3023084
:105CAE0009F0F1C3FE01FF9605A116A127A130A5AB
:105CBE00C8011A2F082D0E94A924F801E35AF44FA7
:105CCE00808391831A2F082D0E94F824882019F4BE
:105CDE000A2F0E94983B01E00093630ED4C326E77F
:105CEE0037E08E010E94B721002341F42DE737E003
:105CFE008E010E94B721002309F43CC1BE01605FF2
:105D0E007F4FE6E6F9E830E08B0148E150E00E9473
:105D1E004644B23071F4FE01FF9605A116A127A1EB
:105D2E0030A5073040E0140740E0240740E0340778
:105D3E0020F002E00E94EF23A6C301E00093630E61
:105D4E00FE01FF9605A116A127A130A5102F07E091
:105D5E000E948E2340E452EE60E070E080E03AC094
:105D6E0002E0809F8001212F220F220B322F040F81
:105D7E00151F261F371F0F5F1F4F2F4F3F4FF80165
:105D8E00322F3BBF069000E00BBF302C222402E0E6
:105D9E00809F8001212F220F220B322F040F151FFF
:105DAE00261F371FF801322F3BBF0690202D00E033
:105DBE000BBF30E0220D331D2F7F3370FE01ED5DE2
:105DCE00FE4F082F10E0000F111FE00FF11F208370
:105DDE0031838395873120F2FE01FF9605A116A12E
:105DEE0027A130A540E450E00E94A543005C1F4F60
:105DFE0080E026C022E0829F000E111E21E0020EDE
:105E0E0020E0121EF001E35AF44F508140E022E0F0
:105E1E00829F000E111EF001E35AF44F208130E0F4
:105E2E00240F351F2F7F3370FE01EB50FF4F482F8D
:105E3E0050E0440F551FE40FF51F208331838395E7
:105E4E008731C0F280E068C0FE01ED5DFE4F082F85
:105E5E0010E0000F111FE00FF11F208131812F7F05
:105E6E0033708E010B501F4FFE01709690E0E80FBD
:105E7E00F91F408150E0440F551F040F151FE02FEE
:105E8E00F12F008111810F7F1370201B310B8E01BA
:105E9E000D5D1E4FFE01709690E0E80FF91F4081D8
:105EAE0050E0440F551F040F151FE02FF12F0081F6
:105EBE0011810F7F1370020F131F22E0829F20E0CB
:105ECE00020E22E0121EF001E35AF44F00831183FA
:105EDE008E010B501F4FFE01709690E0E80FF91FD8
:105EEE00208130E0220F331F020F131FE02FF12FFE
:105EFE000081118100701C7F22E0829F20E0020E43
:105F0E0022E0121EF001E35AF44F20813181202B42
:105F1E00312B208331838395873100F5FE017096F6
:105F2E0090E0E80FF91F00810F3F09F08DCFFE01C1
:105F3E00EB50FF4F082F10E0000F111FE00FF11F65
:105F4E000081118122E0829F20E0020E22E0121ECB
:105F5E00F001E35AF44F00831183DDCF07E00E9476
:105F6E00C12380E0873108F08EC2082F0E94983B33
:105F7E008395F8CF20EC36E08E010E94B7210023E6
:105F8E00E1F111E001E0C8D200E20E948B0D00E2C7
:105F9E000E948B0D00E20E948B0D00E20E948B0D81
:105FAE0080E090E004C0082F0E945F0D01968031C2
:105FBE0000E09007C0F380E090E0803001E09007B1
:105FCE0008F061C2082F0F70002351F40CE810E0A6
:105FDE000E94EF42082F0E94740D0AE30E948B0D5F
:105FEE009C0120503F4FA9010E9487430E94740DCF
:105FFE0000E20E948B0D0196E0CF28EC36E08E0178
:10600E000E94B721002309F457C0B33021F002E0FB
:10601E000E94EF2338C2FE01FF9601A512A523A50B
:10602E0034A5602FFE01FF9605A116A127A130A56C
:10603E00202F30E020503F4F062FA9010E9493439E
:10604E0011E001E069D200E20E948B0D00E20E9495
:10605E008B0D00E20E948B0D00E20E948B0D80E002
:10606E0090E004C0082F0E945F0D0196803100E081
:10607E009007C0F380E090E0803001E0900708F0D8
:10608E0002C2082F0F70002351F40CE810E00E949A
:10609E00EF42082F0E94740D0AE30E948B0D9C01A3
:1060AE0020503F4FA9010E9487430E94740D00E2C9
:1060BE000E948B0D0196E0CF2BEC36E08E010E94F4
:1060CE00B721002389F100E00E94EF230E94350ED4
:1060DE00093519F0093709F0D6C180E090E006C005
:1060EE0000E0FC01E35AF44F00830196803002E099
:1060FE009007B0F300E00093710B00E20093730B76
:10610E0000E20093750B0FEF00936E0B00936B0B79
:10611E0001E00093630E0E94F625A0E08A2E1A2F4E
:10612E00082D0E941324AFC12FEC36E08E010E9481
:10613E00B721002341F424ED36E08E010E94B721F1
:10614E00002309F414C110E0B0E02FEF3FE0A901E5
:10615E000E94874322EF3FE0A9010E94934301E191
:10616E002FEF3FE0A9010E94934380E090E006C02C
:10617E00FC01E35AF44F0081100F0196803002E0CB
:10618E009007B0F300917C0B011B0A9500937C0BDA
:10619E000EE20E948B0D80E090E00BC0FC01E35AF2
:1061AE00F44F00819C012050384FA9010E94934367
:1061BE000196803002E0900788F300919B0D20E05D
:1061CE003AE0A9010E94934300919C0D21E03AE030
:1061DE00A9010E94934380E090E001C001968030B7
:1061EE0002E0900768F49C012050384FA9010E94EC
:1061FE008743FC01E35AF44F1081011779F3B1E0A4
:10620E00E1E6FEE00081118125EF3FE0A9010E9449
:10621E009343BB2309F074C025EF3FE0A9010E9410
:10622E008743E1E6FEE020813181021709F068C064
:10623E000AEA24EF3FE0A9010E94934308E001BD62
:10624E0004EF11E00E94450D25EF3FE0A9010E94E9
:10625E00874310E0E1E6FEE000831183E1E6FEE015
:10626E00008111810F7F107000831183B0E00FEF5A
:10627E0024EF3FE0A9010E949343E1E6FEE0008196
:10628E00118120E030E040E052E060E070E00E94DA
:10629E00E6432801390100E0400E00EE501E00E0FA
:1062AE00601E00E0701E80E090E001C0019680301C
:1062BE0002E09007B8F49C012050384FA9010E94CB
:1062CE008743602F8C0120E030E0040D151D261D44
:1062DE00371DF801322F3BBF069000E00BBF601553
:1062EE0029F3B2E020E03AE0A9010E94874300932F
:1062FE009B0D21E03AE0A9010E94874300939C0D7B
:10630E00BB23F9F40E9421250091720B002361F04A
:10631E00E1E6FEE0008111812091720B30E0205009
:10632E003F4FA9010E94934308ED18E10E94EF42EE
:10633E000E94F625A0E08A2E1A2F082D0E94132403
:10634E0008C008ED16E00E94280EB05D0B2F0E94CB
:10635E008B0D00E00093630E22EF3FE0A9010E9437
:10636E0087432FEF3FE0A9010E9493438CC02DE39A
:10637E0038E08E010E94B721002309F470C091E02D
:10638E00B23039F4FE01FF9605A116A127A130A562
:10639E00902F20E030E010E20EEF0E94760EB0E07B
:1063AE0013C000919B00102F17FF09C00FEF009331
:1063BE00640E0FE41FE00E94EF420E94350E009122
:1063CE00680E002371F7B395B91738F580E018C041
:1063DE00082F10E0F801E255F54F0081002379F007
:1063EE001EE1082F0E944D0E22E0829F20E0020E39
:1063FE0022E0121EF001E35AF44F008311838395BD
:10640E00873130F30EEF0093670E0093640EE1E6D2
:10641E00FEE00081118115D1D2CF08ED18E10E9466
:10642E00EF4280E016C090E0FC01E255F54F00818E
:10643E00002371F01EE1082F43D022E0829F20E05E
:10644E00020E22E0121EF001E35AF44F0083118374
:10645E008395873140F307E00E94C12314C02BEED1
:10646E0037E08E010E94B721002349F019E100E5C3
:10647E0053D0EF966296D395ECE00C94684400E509
:10648E001EE00E94EF420091710B091599F00091E8
:10649E00710B013F20F000E00093710B07C00091DB
:1064AE00710B083018F007E00093710B0E9458240E
:1064BE009090710B1A2F082D0E94BC250C94052765
:1064CE009A938A93802F082F0E944D0E0F3F2FEF25
:1064DE00120719F400E010E81CC0E1E6FEE020818E
:1064EE003181232B51F090E0880F991FFC01E95365
:1064FE00F54F20813181021B130B212F26FF03C084
:10650E0000E010E006C0003024E0120710F00FEF9C
:10651E0013E08991999108959A938A93902F812FE0
:10652E0002E00E948B0D0BE10E948B0D0BE50E9489
:10653E008B0D8A3038F0082F4AE00E949743005D99
:10654E000E948B0D082F4AE00E949743042F005D96
:10655E000E948B0D0BE30E948B0D9A3038F0092FA1
:10656E004AE00E949743005D0E948B0D092F4AE07E
:10657E000E949743042F005D0E948B0D06E60E9439
:10658E008B0D8991999108959A938A93FA93EA9330
:10659E003A922A921A920A927A936A935A934A9349
:1065AE003A932A931A930A938FB79BB700E00BBFC7
:1065BE0078940D9903C00AEF0093660E0091680E51
:1065CE00002309F0BBD0EFE6FEE0008111810F5FE2
:1065DE001F4F008311830091CB0E102F1395109334
:1065EE00CB0E0F700023D1F400916D0E002349F0F5
:1065FE00EDE6FEE000810A95008301E018B3102756
:10660E0018BB00916E0E002349F0EEE6FEE000810D
:10661E000A95008300E813B1102713B99BBF8FBFF3
:10662E0009911991299139914991599169917991CC
:10663E000990199029903990E991F9918991999140
:10664E001895EBE6FEE00083118301E00093690EDE
:10665E0001E00093680E08959A938A930091360E86
:10666E00053018F000E00093360E00916A0E10917E
:10667E00360E011709F45FC080E00091360E10E06F
:10668E000D5F1F4F40E450E00E94A543A80160E05B
:10669E0070E0405C5F416F4F7F4F0CE190E0FC017A
:1066AE00E159F64F0083839502E090E0FC01E15939
:1066BE00F64F0083839500E005C04E5F5F4F6F4F2E
:1066CE007F4F0395073170F510E0F801E255F54F55
:1066DE001081112391F390E0FC01E159F64F0083F4
:1066EE008395FA01362F3BBF069010E01BBF4F5F1C
:1066FE005F4F6F4F7F4F90E0FC01E159F64F0082E4
:10670E008395FA01362F3BBF069010E01BBF4F5FFB
:10671E005F4F6F4F7F4F90E0FC01E159F64F0082C3
:10672E008395CFCF282F13E80EEF0E94D5411091FD
:10673E00360E10936A0E8991999108950E945744CE
:10674E0024970091690E002309F441C000E00093E4
:10675E00851000E010E0EBE7F0E100831183E9E73C
:10676E00F0E100831183EDE7F0E10083118303E094
:10677E0000938310CC2428C002E0C09E80010050FC
:10678E001E4FF801E35AF44F208131810C2D10E099
:10679E00000F111FF801E856F04F2083318300E0FF
:1067AE0010E02C2D30E0220F331FF901E25DFF4E79
:1067BE00008311832C2D30E0220F331FF901E0539B
:1067CE00F14F00831183C39407E1C016A8F2009124
:1067DE008510002369F000913B0A053029F020E076
:1067EE0015E00EEF0E94D54100E00093680E95C7AC
:1067FE00E9E7F0E100811181EBE7F0E120813181E1
:10680E000217130708F045C2E9E7F0E10081118194
:10681E000F5F1F4F0083118300918310033059F4D3
:10682E0000913B0A053009F434C220E015E00EEF6A
:10683E000E94D5412EC220E015E00EEF0E94D541F8
:10684E0080E00EE190E0FC01E159F64F0083839564
:10685E0002E090E0FC01E159F64F00838395CC24D1
:10686E0047C002E0C09E00E0000E02E0101EF001E4
:10687E00E35AF44F20813181203004E0300768F074
:10688E000FEF13E022E0C29E20E0020E22E0121E65
:10689E00F001E35AF44F0083118390E0FC01E159BB
:1068AE00F64FC082839502E0C09E00E0000E02E02B
:1068BE00101EF001E35AF44F0081118190E0FC01AB
:1068CE00E159F64F0083839502E0C09E00E0000E72
:1068DE0002E0101EF001E35AF44F00811181012FE6
:1068EE0010E090E0FC01E159F64F00838395C394CC
:1068FE0007E1C01608F0C8C1DD24F601E255F54FD8
:10690E0000810023A1F300918310002309F092C0AF
:10691E000C2D10E0000F111FF801E653F04F00810F
:10692E0011812C2D30E0220F331FF901E450F04F6E
:10693E0020813181021B130B212F220F220B322FAC
:10694E00E9E7F0E14081518160E070E00E94E643AA
:10695E00EBE7F0E14081518160E070E00E9430444D
:10696E002C2D30E0220F331FF901E450F04F4081FF
:10697E005181400F511F2C2D30E0220F331FF90192
:10698E00E25DFF4E408351832C2D30E0220F331FEA
:10699E00F901E450F04F2081318115950795020FD2
:1069AE00131F212F220F220B322FE9E7F0E1408136
:1069BE00518160E070E00E94E64340E950E060E003
:1069CE0070E00E94E6434FE050E060E070E00E940D
:1069DE003044012F122F232F330F330B259517958C
:1069EE0007952C2D30E0220F331FF901EC5CF04F90
:1069FE00008311830C2D10E0000F111FF801EA59CE
:106A0E00F04F208131810C2D10E0000F111FF80185
:106A1E00EC5CF04F00811181020F131F22E0C29E29
:106A2E0020E0020E22E0121EF001E35AF44F008322
:106A3E00118310C100918310013009F046C00C2D56
:106A4E0010E0000F111FF801EA59F04FA081B1813B
:106A5E000C2D10E0000F111FF801EE5FF04F0081BA
:106A6E001181212F220F220B322FE9E7F0E1408115
:106A7E00518160E070E00E94E643EBE7F0E1408177
:106A8E00518160E070E00E9430440A0F1B1F22E02B
:106A9E00C29E20E0020E22E0121EF001E35AF44FD5
:106AAE00008311830C2D10E0000F111FF801E65327
:106ABE00F04F208131810C2D10E0000F111FF801D5
:106ACE00E25DFF4E20833183C5C0DD24F601E05A1E
:106ADE00FF4E0081002309F078C00C2D10E0000F4E
:106AEE00111FF801E450F04F0081118111950195AD
:106AFE001040212F220F220B322FE9E7F0E14081C7
:106B0E00518160E070E00E94E643EBE7F0E14081E6
:106B1E00518160E070E00E9430442C2D30E0220F55
:106B2E00331FF901E450F04F40815181400F511F46
:106B3E002C2D30E0220F331FF901E25DFF4E408312
:106B4E0051832C2D30E0220F331FF901EA59F04FFB
:106B5E00A081B1812C2D30E0220F331FF901E450BA
:106B6E00F04F2081318115950795020F131F212FAC
:106B7E00220F220B322FE9E7F0E14081518160E0D4
:106B8E0070E00E94E64340E950E060E070E00E9451
:106B9E00E6434FE050E060E070E00E943044012F89
:106BAE00122F232F330F330B2595179507950A0FA9
:106BBE001B1F22E0C29E20E0020E22E0121EF001F8
:106BCE00E35AF44F0083118345C00C2D10E0000FE3
:106BDE00111FF801EA59F04FA081B1810C2D10E080
:106BEE00000F111FF801EE5FF04F00811181212F70
:106BFE00220F220B322FE9E7F0E14081518160E054
:106C0E0070E00E94E643EBE7F0E14081518160E0E5
:106C1E0070E00E9430440A0F1B1F22E0C29E20E04B
:106C2E00020E22E0121EF001E35AF44F008311838C
:106C3E000C2D10E0000F111FF801E653F04F2081CC
:106C4E0031810C2D10E0000F111FF801E25DFF4E97
:106C5E002083318302E0C09E00E0000E02E0101E91
:106C6E00F001E35AF44F018106FFFBCD00E010E086
:106C7E0022E0C29E20E0020E22E0121EF001E35A34
:106C8E00F44F0083118309CE282F14E80EEF0E94D3
:106C9E00D541E9E7F0E100811181EBE7F0E12081D8
:106CAE0031810217130708F438C500E010E0E9E758
:106CBE00F0E100831183CC2427C002E0C09E00E0E7
:106CCE00000E02E0101EF001E35AF44F20813181D4
:106CDE000C2D10E0000F111FF801EA59F04F208320
:106CEE0031830C2D10E0000F111FF801E25DFF4EF5
:106CFE00208131810C2D10E0000F111FF801E4509E
:106D0E00F04F20833183C39407E1C016B0F2009197
:106D1E008310002309F09FC001E000938310EFE77A
:106D2E00F0E100811181E1E8F0E120813181220F53
:106D3E00331F021B130BEBE7F0E100831183CC240E
:106D4E0046C00C2D10E0000F111FF801E053F14F5B
:106D5E00808191810C2D10E0000F111FF801EC5C69
:106D6E00F04F00811181801B910B0C2D10E0000F54
:106D7E00111FF801E653F04F00811181212F220FD0
:106D8E00220B322FE1E8F0E14081518160E070E0AA
:106D9E000E94E6434CE050E060E070E00E94E64363
:106DAE0045E050E060E070E00E943044012F122F69
:106DBE00232F330F330B801B910B0C2D10E0000F84
:106DCE00111FF801EE5FF04F80839183C39407E1AA
:106DDE00C01608F09FC0DD24F601E05AFF4E008178
:106DEE00013009F0AECF0C2D10E0000F111FF8018D
:106DFE00E053F14F008111812C2D30E0220F331F13
:106E0E00F901EC5CF04F20813181021B130B212F15
:106E1E00220F220B322FEBE7F0E14081518160E02F
:106E2E0070E00E94E643EFE7F0E140815181E1E836
:106E3E00F0E160817181461B570B60E070E00E94AB
:106E4E0030442C2D30E0220F331FF901EE5FF04F4E
:106E5E0000831183BBCF009183100130D1F502E086
:106E6E0000938310E1E8F0E100811181EBE7F0E19E
:106E7E0000831183CC2407E1C01608F04BC00C2D03
:106E8E0010E0000F111FF801E053F14F2081318106
:106E9E000C2D10E0000F111FF801EE5FF04F008176
:106EAE001181201B310B0C2D10E0000F111FF8016A
:106EBE00EC5CF04F00811181201B310B0C2D10E08A
:106ECE00000F111FF801EE5FF04F20833183C39442
:106EDE00D2CF009183100230B1F4EDE7F0E10081E2
:106EEE001181012B61F003E000938310EDE7F0E1D7
:106EFE0000811181EBE7F0E1008311830BC000E00C
:106F0E000093831007C000918310033019F400E042
:106F1E000093831000918310002309F0FEC3E4E870
:106F2E00F0E1008103950083009184101091330EDF
:106F3E00011728F40091690E002309F4D3C00091C3
:106F4E00690E0023A9F50091670E10913B0E0117F3
:106F5E0041F400913A0E10E0EBE6FEE0008311835F
:106F6E0023C00091670E10913D0E011741F4009160
:106F7E003C0E10E0EBE6FEE00083118315C000919D
:106F8E00670E1091640E011741F00091390E10E05A
:106F9E00EBE6FEE00083118307C00091380E10E08F
:106FAE00EBE6FEE0008311830091670E0093640E02
:106FBE00EBE6FEE000811181012B21F401E000934C
:106FCE00851090C000E00093690EE1E6FEE00081BE
:106FDE001181EBE6FEE0208131810217130719F5CE
:106FEE0000E010E020E030E0ECECFEE000831183E6
:106FFE0022833383ADE0B0E0A03400E0B00708F0A8
:10700E0047C0ECECFEE000811181228133810A0F32
:10701E001B1FF801E35AF44F0081FD01E15EF14FB1
:10702E0000831196E9CFEBE6FEE00081118120E0AE
:10703E0030E040E052E060E070E00E94E643005035
:10704E0010422F4F3F4FECECFEE000831183228362
:10705E003383ADE0B0E018C0ECECFEE0408151812E
:10706E00628173818D0120E030E0040F151F261F11
:10707E00371FF801322F3BBF069000E00BBFFD011A
:10708E00E15EF14F00821196A03400E0B00720F3CC
:10709E00ECECFEE00081118122813381005C1F4FF8
:1070AE002F4F3F4F0083118322833383D5DA009114
:1070BE00330E083020F40091330E002381F402E6E3
:1070CE001DE00E94EF42EBE6FEE0008111810E947E
:1070DE000B0E0DE50E948B0D01E00093851000E074
:1070EE0000938410A0E0B0E020C0ECECFEE0008144
:1070FE00118122813381A801B9014F5F5F4F6F4F1C
:10710E007F4FECECFEE04083518362837383F80182
:10711E00322F3BBF069000E00BBF8D01005C1D4F70
:10712E00F801E35AF44F00821196A03400E0B00744
:10713E0058F5E1E6FEE000811181EBE6FEE02081EC
:10714E0031810217130789F6ECECFEE00081118104
:10715E0022813381F801E35AF44F20818D01005CC6
:10716E001D4FF801E35AF44F2083ECECFEE0008152
:10717E001181228133810F5F1F4F2F4F3F4F0083AD
:10718E00118322833383D0CF009184100395EBE6D5
:10719E00FEE0808191811091330E011788F10091EC
:1071AE00670E10913B0E011719F480913A0E14C020
:1071BE000091670E10913D0E011719F480913C0E4F
:1071CE000BC00091670E1091640E011719F080919B
:1071DE00390E02C08091380E082F10E020E030E00A
:1071EE0040E052E060E070E00E94E643005C1F4128
:1071FE002F4F3F4FECECFEE000831183228333834D
:10720E00A0E0B0E01BC0ECECFEE040815181628159
:10721E0073818D0120E030E0040F151F261F371FEC
:10722E00F801322F3BBF069000E00BBF8D010058D6
:10723E001D4FF801E35AF44F00821196A03400E07E
:10724E00B007D0F4E1E6FEE0008111818017D9F697
:10725E00ECECFEE000811181228133810A0F1B1FAD
:10726E00F801E35AF44F20818D0100581D4FF801AB
:10727E00E35AF44F2083E1CF00918510002309F0EB
:10728E004CC20091DB0D10E045E00E94B5434091E9
:10729E00350E50E00E94C143EDE7F0E1008311830B
:1072AE000091DC0D1091350E019F800145E00E948A
:1072BE00BB43D8010A2F0B2B11F4A8E0B0E000E07D
:1072CE0010E0CC240EC02C2D30E0220F331FF9011C
:1072DE00E053F14F208131810217130708F4890121
:1072EE00C39427E1C21608F0DEC0DD24F601E25594
:1072FE00F54F20812223A1F32C2D30E0220F331FD6
:10730E00F901E856F04F4081518122E0C29E20E003
:10731E00020E22E0121EF001E35AF44F4083518315
:10732E002C2D30E0220F331FF901EA59F04F408324
:10733E00518322E0C29E20E4020E22E0121EF001D2
:10734E00E35AF44F208131812F7F33704C2D50E062
:10735E00440F551FFA01E953F54F40815181240F17
:10736E00351F432F46FF03C020E030E006C020301B
:10737E0044E0340710F02FEF33E04C2D50E0440F73
:10738E00551FFA01E856F04F40815181B901641B37
:10739E00750B4C2D50E0440F551FFA01E053F14F81
:1073AE00608371834C2D50E0440F551FFA01E8564F
:1073BE00F04F608171814C2D50E0440F551FFA0142
:1073CE00E856F04F2083318342E0C49E40E8040E1D
:1073DE0042E0141EF001E35AF44F008011804FEF8B
:1073EE00042243E014224C2D50E0440F551FFA01A5
:1073FE00E953F54F40815181400D511D052E06FE7A
:10740E0003C040E050E006C04030E4E05E0710F0FC
:10741E004FEF53E06217730718F42417350730F057
:10742E002617370728F44217530710F420E001C03F
:10743E0021E0222391F4EDE7F0E120813181232B2D
:10744E0061F42091841030E0E091330EF0E031973A
:10745E002E173F074CF0882339F420E0DD24F60187
:10746E00E05AFF4E208306C021E0DD24F601E05AEB
:10747E00FF4E20832C2D30E0220F331FF901E053F5
:10748E00F14F4081518155230AF01DCF2C2D30E054
:10749E00220F331FF901E053F14F208131813195D5
:1074AE002195304019CF48E250E00E94A543C80113
:1074BE008D0143E050E00E94A543A8018C010E947B
:1074CE00C143EFE7F0E1008311830091370E10E026
:1074DE00E1E8F0E100831183E1E8F0E10081118140
:1074EE00000F111FEFE7F0E1208131810217130722
:1074FE0080F10091A90A002399F00BE50E948B0DF3
:10750E00009184100E94740D0CE20E948B0DEFE727
:10751E00F0E1008111810E940B0E0DE50E948B0D92
:10752E00EFE7F0E100811181012B39F400E010E06A
:10753E00E1E8F0E1008311830CC0EFE7F0E1008198
:10754E0011810150104016950795E1E8F0E1008396
:10755E001183EFE7F0E10081118120E030E0000FB0
:10756E00111F221F331FE1E8F0E180819181A0E01D
:10757E00B0E0880F991FAA1FBB1F081B190B2A0BFF
:10758E003B0B48015901880C991CAA1CBB1C880E88
:10759E00991EAA1EBB1E000F111F221F331F088328
:1075AE0019832A833B83082D09290A290B2929F4DB
:1075BE009924AA24BB2488248394088119812A81C2
:1075CE003B81012B022B032B41F401E010E020E064
:1075DE0030E0088319832A833B83CC2442C00419EC
:1075EE00150926093709A401B5010E9430442C2D36
:1075FE0030E0220F331FF901E653F04F0083118361
:10760E000C2D10E0000F111FF801E653F04F2081F2
:10761E003181203004E030075CF00FEF13E02C2DA9
:10762E0030E0220F331FF901E653F04F0083118330
:10763E000C2D10E0000F111FF801E653F04F2081C2
:10764E00318121300CEF30075CF401E01CEF2C2D62
:10765E0030E0220F331FF901E653F04F0083118300
:10766E00C39407E1C01608F050C00C2D10E0000FB7
:10767E00111FF801E450F04F00811181212F220FCC
:10768E00220B322FAC01BD010E94E64328013901C5
:10769E000C2D10E0000F111FF801E053F14F008187
:1076AE001181212F220F220B322F0801190140E0E8
:1076BE005AE060E070E0800191010E94E64308010B
:1076CE0019014CE050E060E070E0800191010E94F1
:1076DE003044DD24F601E05AFF4E4081442309F088
:1076EE007ECF0419150926093709488159816A8107
:1076FE007B810E9430442C2D30E0220F331FF90184
:10770E00E653F04F008311837BCFE1E8F0E1008177
:10771E001181EBE7F0E1008311832496EEE00C94E7
:10772E00664410E0F801E255F54F1081112309F47B
:10773E005DC012E0019F10E0010E12E0111EF0017B
:10774E00E35AF44F118117FF05C020E018E10E94A3
:10775E006D0E0895E1E6FEE020813181232BC9F004
:10776E0012E0019F10E0010E12E0111EF001E35A2B
:10777E00F44F408151814F7F5370202F30E0220F04
:10778E00331FF901E953F54F20813181240F351F45
:10779E000DC012E0019F10E0010E12E0111EF0016B
:1077AE00E35AF44F208131812F7F3370132F16FF50
:1077BE0003C020E030E006C0203014E0310710F0A6
:1077CE002FEF33E01EE110936F09122F1093700903
:1077DE00232F30E02093710910E51093720910E009
:1077EE001093730925E013E00E94D54108959A93F2
:1077FE008A9390E080E014C020E0082F10E0F8019A
:10780E00E255F54F208320E030E802E0809F8001B2
:10781E0000501E4FF801E35AF44F208331838395B5
:10782E008731E8F5EEEEF8E1082F10E0E00FF11FDA
:10783E000491002309F320E011E0082F0E94514229
:10784E000023C1F02FEF082F10E0F801E255F54F9D
:10785E00208314E2082F0E944D0E22E0829F20E02A
:10786E00020E22E0121EF001E35AF44F0083118340
:10787E009395D5CF20E0082F10E0F801E255F54F93
:10788E00208300E010E822E0829F20E0020E22E03A
:10789E00121EF001E35AF44F00831183C0CF40EC67
:1078AE0050EE60E070E080E048C002E0809F800112
:1078BE00212F220F220B322F040F151F261F371FC9
:1078CE000F5F1F4F2F4F3F4FF801322F3BBF0690D8
:1078DE00102D00E00BBF00E022E0829F212C220C35
:1078EE002208322C040E151E261E371EF001322DD4
:1078FE003BBF069020E02BBF1124000E111E082F57
:10790E0010E0000F111FF801E953F54F00821182AC
:10791E0000E010E0282F30E0220F331FF901E7506E
:10792E00F54F00831183282F30E0220F331FF9010A
:10793E00E55DF44F008311838395873108F4B5CF4D
:10794E00092F8991999108952091670E2093640EC5
:10795E0020E030E0E1E6FEE0208331830E94283310
:10796E0001C005D00091680E0023D9F7089500914B
:10797E00720E063018F000E00093720E00917C0E2D
:10798E0010917B0E0117F9F000917C0E10E00F7034
:10799E001070F801E358F14F0081ECE7FEE0108122
:1079AE00139510830F3F19F410E01093720E20916F
:1079BE00720E30E0F901ED58F14F0083E2E7FEE080
:1079CE000081039500830091720E063009F066C0A7
:1079DE000091770E1091780E2091730E2F3F09F0C3
:1079EE0054C02091740E253509F04FC02091750EAC
:1079FE000095201709F049C00091760E10950117D9
:107A0E0009F043C00091750E0093650E0091760E3D
:107A1E000093660E0091650E0F3329F420E018E1F5
:107A2E000EEF0E946D0E0091650E003821F400E8F5
:107A3E000093670E26C000916E08013029F4009164
:107A4E00650E0093670E1DC000916E08023031F472
:107A5E000091650E005C0093670E13C000916E08D6
:107A6E00043031F40091650E00580093670E09C082
:107A7E0000916E08083029F40091650E00540093B1
:107A8E00670E01E00093710E089500916E0E0430A2
:107A9E0028F4EEE6FEE000810E5F008308950FEFFE
:107AAE0010E0E1E6FEE000831183F89421E012E29B
:107ABE0001E00E94110D00E000937B0E00937C0EFE
:107ACE00789401E000936E0800E80093670E1E9A0A
:107ADE001C9A1B9802C0C09A1F9A0091660E0A3F0C
:107AEE00C9F41E980D9BFECF04E610E00E94450DD2
:107AFE0000E00093660E77D00091660E0A3FD9F72C
:107B0E001E9A0D9BFECF04E610E00E94450D00E08C
:107B1E000093660E2CDF0091710E0130F1F600E03D
:107B2E000093710E0091650E0F700F3029F420E056
:107B3E0018E10EEF0E946D0E1091650E1F700091F0
:107B4E00650E003841F22091670E30E020503F4F15
:107B5E00A9010E9487432091650E2073203309F5F9
:107B6E00C0981F98113031F41E9A1C9A1B981093CE
:107B7E006E0817C0123031F41E9A1C981B98109381
:107B8E006E080FC0143031F41E981C981B98109379
:107B9E006E0807C0183029F41E9A1C9A1B9A10936F
:107BAE006E08112309F499CF013028F0003818F42B
:107BBE0010E0CADE92CF00916D0E083008F08DCF26
:107BCE00EDE6FEE000810C5F008387CF18E20E9495
:107BDE004D0E013024E012072CF000501440119588
:107BEE000195104008950E945C4480E090E03C01B5
:107BFE002C01DC0188241BC002E1E8DF800F911FFD
:107C0E0003E1E4DF801B910B05E1E0DF400E511E26
:107C1E0004E1DCDF601A710A06E1D8DFA00FB11FA4
:107C2E00882021F404E610E00E94450D839402E0C2
:107C3E00801610F3A13800E0B0074CF0E6E8F0E152
:107C4E00008100FF04C004E010E07EDEB1C0A13868
:107C5E0000E0B0075CF000918610002339F403E0D9
:107C6E0010E072DE01E000938610A2C0A0380FEF84
:107C7E00B0074CF4E6E8F0E1008101FF04C006E035
:107C8E0010E062DE95C0A0380FEFB0075CF40091F3
:107C9E008610002339F405E010E056DE02E0009372
:107CAE00861086C0813002E090074CF0E6E8F0E1E5
:107CBE00008104FF04C008E010E046DE79C0813088
:107CCE0002E090075CF000918610002339F407E083
:107CDE0010E03ADE00E1009386106AC080300EEFAD
:107CEE0090074CF4E6E8F0E1008105FF04C00AE0DD
:107CFE0010E02ADE5DC080300EEF90075CF400913C
:107D0E008610002339F409E010E01EDE00E2009335
:107D1E0086104EC001E0401601E050064CF0E6E839
:107D2E00F0E1008103FF04C00EE010E00DDE40C064
:107D3E0001E0401601E050065CF000918610002331
:107D4E0039F40DE010E000DE08E00093861030C03C
:107D5E0001E0601601E070064CF0E6E8F0E100810B
:107D6E0002FF04C00CE010E0EFDD22C001E060165F
:107D7E0001E070065CF000918610002339F40BE0F0
:107D8E0010E0E2DD04E00093861012C0A82BB92BA0
:107D9E00A429B529A629B729AB2B51F40091861039
:107DAE00002331F001E010E0CFDD00E000938610FB
:107DBE0002E310E00E94450DE9E00C946B440E9432
:107DCE005B441A980E94F00C00E00093A70A0093FF
:107DDE00A80A0FEF13E0ECEAFAE00083118300E04B
:107DEE000093A90A0093AA0A00E00093680E0FEF11
:107DFE0000936A0E00E80093670E23EF3FE0A9019F
:107E0E000E948743802E05E1802E22E030E0A901FA
:107E1E000E9487430F3F39F021E030E0A9010E9414
:107E2E0087430F3FD1F401E000939C0A21E030E03C
:107E3E00A9010E94934302E200939B0A20E030E0E6
:107E4E00A9010E94934300E022E030E0A9010E94C4
:107E5E00934305E00E94BE0C0EC021E030E0A90164
:107E6E000E94874300939C0A20E030E0A9010E9403
:107E7E00874300939B0A11E020E830E000E00E9467
:107E8E009F0C21E010919B0A00E00E94110D20E052
:107E9E0012E201E00E94110D00E00093A70A009388
:107EAE00A80A24EF3FE0A9010E948743053519F483
:107EBE0078949DDC55C180E013C01E981C981B98C9
:107ECE00C0981F9804E610E00E94450D1E9A1C9A59
:107EDE001B9AC09A1F9A04E610E00E94450D8395E6
:107EEE00823058F300E910E073D33BD325E030E045
:107EFE00A9010E948743013189F40DE91EE068D380
:107F0E0080E00AC0282F30E0205C3F4FA9010E947C
:107F1E0087430E948B0D83958C30A0F3789403E1F8
:107F2E00801609F46DD106E18016E9F500E1402EC8
:107F3E005524662477240AEB11E04AD32FC0009112
:107F4E00A80A1091A70A0117B1F080E090E0A0E016
:107F5E00B0E099240091A80A10E0F801E159F74F1A
:107F6E000081E8EAFAE01081139510830E94740DE7
:107F7E0000E20E948B0D8F5F9F4FAF4FBF4F841556
:107F8E009505A605B705D8F2992041F40DE00E949B
:107F9E008B0D0AE00E948B0D9924939480E090E063
:107FAE00A0E0B0E0ECCF04E1801631F401E00093E4
:107FBE00A90A0E94840EFDCF00919B0A013061F147
:107FCE0001E000939B0A20919B0A14E00EEF0E94A1
:107FDE00640E0AE912E0FCD200E814E82EE130E06B
:107FEE0040919B0A50E060E070E04F5F5F4F6F4F33
:107FFE007F4F0E9430440E94B20D06EB12E0E8D291
:10800E0000919B0A20E030E0A9010E94934309B938
:10801E0008EE13E00E94450DEADB002309F04CC088
:10802E0002E200939B0A20919B0A14E00EEF0E943D
:10803E00640E0AE912E0CCD200E814E82EE130E03A
:10804E0040919B0A50E060E070E04F5F5F4F6F4FD2
:10805E007F4F0E9430440E94B20D06EB12E0B8D260
:10806E0001E000939B0A20919B0A14E00EEF0E9400
:10807E00640E0AE912E0ACD200E814E82EE130E01A
:10808E0040919B0A50E060E070E04F5F5F4F6F4F92
:10809E007F4F0E9430440E94B20D06EB12E098D240
:1080AE0000919B0A20E030E0A9010E94934309B998
:1080BE0008EE13E00E94450D01E00093A90AA3D239
:1080CE0000E010E0E1E6FEE0008311830E9421252E
:1080DE0080E016C090E0FC01E255F54F00810023D0
:1080EE0071F014E2082F0E944D0E22E0829F900143
:1080FE0020503E4FF901E35AF44F008311838395CC
:10810E00873140F30091710B023049F00CEC1EE008
:10811E005FD220E018E10EEF0E946D0E0EC00D9999
:10812E0009C003EB1EE054D220E018E10EEF0E94CE
:10813E006D0E03C001E010E007DC20E030E010E23D
:10814E000EEF0E94760E02E1801679F001E010E04B
:10815E00E1E6FEE0008311830E9421250E94F625B0
:10816E0001E00093A90A0E94E02600E00093A90A0C
:10817E0096DCECCFFA93EA934A933A932A931A93A6
:10818E000A933FB74BB700E00BBF20919C000091C4
:10819E007B0E10E00F701070F801E358F14F208342
:1081AE00EBE7FEE00081039500834BBF3FBF0991D3
:1081BE001991299139914991E991F9911895FA936B
:1081CE00EA934A933A932A931A930A933FB74BB77B
:1081DE0000E00BBF0091A70A102F13951093A70A6A
:1081EE002CB110E0F801E159F74F20834BBF3FBF90
:1081FE0009911991299139914991E991F99118951E
:10820E001E981C9806EA10E0E3D121C00E94350E9C
:10821E000E94870D5E9A00919B00102F17FDF6CFDE
:10822E005E9BFECF1A980091A80A1091A70A01171B
:10823E0071F00091A80A10E0F801E159F74F0081A2
:10824E00E8EAFAE01081139510830E948B0D0091DD
:10825E009B00102F17FFE7CF1A9ADDCF0E946144C3
:10826E00902F002480E013C00091A80A10E0F801BE
:10827E00E159F74F0081E8EAFAE010811395108377
:10828E00282F30E0F901ED52F64F008383958917C0
:10829E00F0F400E010E020E030E04091A80A5091A8
:1082AE00A70A451791F4A801B9018A019B010F5F36
:1082BE001F4F2F4F3F4F4133E5E75E07E0E06E075C
:1082CE00E0E07E0750F300240394002069F2A82F0B
:1082DE00B0E00091390A0E3F09F45CC00091A90A82
:1082EE00002309F457C0002049F09F3F39F006E7FC
:1082FE001DE06ED10091A70A0093A80AA43008F4DD
:10830E0049C00091D3090F3F21F40091D4090F3FCA
:10831E0049F00DE81DE05CD10091A70A0093A80A70
:10832E0000E039C00091D5091091390A011749F0C2
:10833E0005EA1DE04DD10091A70A0093A80A00E0BE
:10834E002AC02091D60930E00A2F10E004501040C8
:10835E002017310749F00DEB1DE03AD10091A70A25
:10836E000093A80A00E017C082E007C090E0FC016D
:10837E00ED52F64F0081B00F83958A17B8F3BF3FC9
:10838E0049F005ED1DE024D10091A70A0093A80A3B
:10839E0000E001C00A2FE4E00C9470440E94614496
:1083AE003FEF3093370A3FEF3093380A0093390A84
:1083BE00022F0E5F00933A0A10933B0A80E00DC025
:1083CE0090E0FC01E159F64F0081A82FB0E0159620
:1083DE00FD01E95CF54F00838395821788F300E079
:1083EE002A5FA22F82E007C090E0FC01E95CF54F06
:1083FE001081010F839590E0EA2FF0E031978E17F0
:10840E009F0794F3009590E0FC01E95CF54F008323
:10841E001A9A80E009C05E9A90E0FC01E95CF54F83
:10842E0000810E94870D83958A17A8F35E9BFECF6D
:10843E001A980A2FE4E00C9470440E946144D8010B
:10844E00922F992359F40091390A0E3F21F40AEE26
:10845E0011E0BED003C00BE012E0BAD080E00CC039
:10846E00082F10E0FD01E00FF11F00810E94740D36
:10847E0000E20E948B0D8395891790F30BE312E0B7
:10848E00A7D0092F0E94930D09E20E948B0DE4E004
:10849E000C9470440E945F44502E912FB22FA0E096
:1084AE000EC000916E0E0A3028F4EEE6FEE000815A
:1084BE000E5F00830091A70A0093A80AA395A3302C
:1084CE00B0F42B2F192F052D69DF802F923029F450
:1084DE004090700906E0400E02C006E0402E042DCA
:1084EE00BDDE0093AB0A0091AB0A0415D1F60091E4
:1084FE00AB0A0415F9F00091390A0E3FD9F000913C
:10850E00A90A0023A9F003E41EE062D0052D0E9403
:10851E00740D05EB10E05CD0282F07E31AE08DDF19
:10852E0007EC10E055D02091AB0A03ED19E085DF82
:10853E0000E014C00091AA0A002379F005EB10E0C8
:10854E0047D0282F07E31AE078DF07EC10E040D081
:10855E002091AB0A03ED19E070DF01E0E6E00C9428
:10856E006E4409ED10E034D000E814E82EE130E05E
:10857E004091990050E060E070E04F5F5F4F6F4FA9
:10858E007F4F0E9430440E94B20D00E20E948B0D7C
:10859E0006EB12E01DD00CE20E948B0D03EE10E0F4
:1085AE0017D000E814E82EE130E049B150E060E069
:1085BE0070E04F5F5F4F6F4F7F4F0E9430440E94BD
:1085CE00B20D00E20E948B0D06EB12E001D0089571
:1085DE00EF97EF97A49720E001C02395203A60F41F
:1085EE0030E0F801E20FF31F4491FE0130E0E20F9C
:1085FE00F31F4083442389F78E010E94280EEF96C5
:10860E00EF96A49608959A938A930CE21DE0E0DF0C
:10861E0090E080E007C00DE20E948B0D0DE50E94F8
:10862E008B0D83958731B0F40BE50E948B0D082FCF
:10863E000E94740D0AE30E948B0D082F10E0F801C2
:10864E00E255F54F0081002331F30FE40E948B0DAC
:10865E009395E4CF0DE31DE0BBDF092F0E94740D4F
:10866E0008E20E948B0D092F0E94930D09E20E94D1
:10867E008B0D03E41DE0ACDF07E10E94740D08E2F0
:10868E000E948B0D07E10E94930D09E20E948B0D53
:10869E0080E013C090E0FC01E255F54F008100230D
:1086AE0059F015E0082F0E943D0E002329F020E01E
:1086BE0015E0082F0E946D0E8395873158F389912E
:1086CE00999108950FEB0DBF06E00EBFC0E8D6E0FE
:1086DE000E947B44002311F00E948D4400E00BBFEA
:1086EE000E94E63E0E94B0440C94B044E199FECF45
:1086FE0008954F5F5F4FFADF4EBB5FBBE09A089560
:10870E00FADF0DB308954F5F5F4F4EBB5FBBF8941A
:10871E00E29AE19A0FBE08950FB6E8DF0DBBF5CFD2
:10872E000024E8E0EA9532F0001F001C0416D0F396
:10873E00041AF8CF001F402D00950895002411242F
:10874E000030010741F01695079510F4040E151E22
:10875E00440F551FF5CF002D112D08954A951AF08F
:10876E00000F111FFBCF08954A951AF01695079525
:10877E00FBCF089500241124EFE0001F111F001CF1
:10878E00111C0416150610F0041A150AEA95AAF71C
:10879E00001F111F402D512D0095109508953095F5
:1087AE002095109501951F4F2F4F3F4F08957095AF
:1087BE006095509541955F4F6F4F7F4F0895002400
:1087CE00112422243324E02FE12BE22BE32B71F032
:1087DE00369527951795079520F4040E151E261E1F
:1087EE00371E440F551F661F771FEDCF002D112D1D
:1087FE00222D332D08954A952AF0000F111F221FA6
:10880E00331FF9CF08950024112422243324E0E2EB
:10881E00EA9592F0001F111F221F331F001C111C1E
:10882E00221C331C041615062606370688F3041A76
:10883E00150A260A370AECCF001F111F221F331FFD
:10884E00402D512D622D732D00951095209530954C
:10885E000895FF2777231AF4F1600E94DE43332335
:10886E001AF4F0950E94D6430E940A44F69510F42D
:10887E000E94D643F69510F40C94DE430895AF9300
:10888E00BF93B12FA02F3BBFD895EF5FFF4F3F4F48
:10889E000D9241505040B9F74BBFBF91AF91089523
:1088AE00DA92CA92BA92AA929A928A927A926A921A
:1088BE005A924A92BA93AA939A938A930895DD8410
:1088CE00CC84BB84AA84998488847F806E805D80EA
:1088DE004C80BB81AA8199818881F0E00FB6F89413
:1088EE00CE0FDF1F0FBE089501E0089520E002D0E5
:1088FE00E9F708952D9301501040202F212B089554
:10890E003BBF27913BB7F6DFD9F7089509EA19E87F
:10891E002801F20130E03BBF07911691F201329629
:10892E00A791B691F2013496479157916691242FF3
:10893E00252B262B21F0FA01362FE2DF01C0D6DFE0
:10894E0007E0400E00E0501EA201473B594808F3D5
:10895E00089500008895FECF00FF03020504070668
:10896E0009080B0A0D0C0F0E111013121514160018
:10897E00080808090909090909090909090909095C
:10898E00090909090808080707151B20252A2F348D
:10899E0039141A1F24292E33383D4DAF01C006B7A6
:1089AE00890018086F0800000052454D4F434F4E86
:1089BE00005257004E4557005341564500534156FD
:1089CE000020457272004D4F54494F4E20376600BD
:1089DE004845580048005245414400524400520058
:1089EE0043414C440043414C550053575200535998
:1089FE004E435F575200575249544500575200524A
:108A0E0045004D4F4E00474F544F004E45585400B1
:108A1E004E004245464F52450042005041474500E8
:108A2E00434F5059004E414D45004F4E004F464664
:108A3E0000535445500053004D4F56004D4F564570
:108A4E000044454C45544500494E53455254004947
:108A5E004E4954004D4F54494F4E00534554004D0E
:108A6E004952524F52004D004545505F55500045FA
:108A7E0045505F444E0055504441544500534341C8
:108A8E004E004C4544005345415243480042415527
:108A9E0044004D4F4E49544F520044454D4F0043F4
:108AAE00484B005445535400434944000D0A205B83
:108ABE004349443A3078005D2000535953005359CE
:108ACE005354454D000D0A2042616420436F6D6D75
:108ADE00616E6400455849540048454C500054009E
:108AEE00544F53530057005245475F575200525749
:108AFE005200414354494F4E004143540053595381
:108B0E005F5752005245534554000D0A205B5245A3
:108B1E005345545D0044524553455400474F00475A
:108B2E000050494E4700504C4159005000494400F6
:108B3E00490042545F424155440042545F52440042
:108B4E00425400424C5545544F4F54480044554DE5
:088B5E005000440055500001D5
:00000001FF
